******************************************************************************
                  MSP430 Linker PC v4.4.4                      
******************************************************************************
>> Linked Mon Jul 13 22:09:50 2015

OUTPUT FILE NAME:   <ADS1262_TIPD188.out>
ENTRY POINT SYMBOL: "_c_int00_noargs"  address: 0000461a


MEMORY CONFIGURATION

         name            origin    length      used     unused   attr    fill
----------------------  --------  ---------  --------  --------  ----  --------
  SFR                   00000000   00000010  00000000  00000010  RWIX
  PERIPHERALS_8BIT      00000010   000000f0  00000000  000000f0  RWIX
  PERIPHERALS_16BIT     00000100   00000100  00000000  00000100  RWIX
  INFOD                 00001800   00000080  00000000  00000080  RWIX
  INFOC                 00001880   00000080  00000000  00000080  RWIX
  INFOB                 00001900   00000080  00000000  00000080  RWIX
  INFOA                 00001980   00000080  00000000  00000080  RWIX
  USBRAM                00001c00   00000800  00000000  00000800  RWIX
  RAM                   00002400   00002000  00000b24  000014dc  RWIX
  FLASH                 00004400   0000bb80  00005a59  00006127  RWIX
  INT00                 0000ff80   00000002  00000000  00000002  RWIX
  INT01                 0000ff82   00000002  00000000  00000002  RWIX
  INT02                 0000ff84   00000002  00000000  00000002  RWIX
  INT03                 0000ff86   00000002  00000000  00000002  RWIX
  INT04                 0000ff88   00000002  00000000  00000002  RWIX
  INT05                 0000ff8a   00000002  00000000  00000002  RWIX
  INT06                 0000ff8c   00000002  00000000  00000002  RWIX
  INT07                 0000ff8e   00000002  00000000  00000002  RWIX
  INT08                 0000ff90   00000002  00000000  00000002  RWIX
  INT09                 0000ff92   00000002  00000000  00000002  RWIX
  INT10                 0000ff94   00000002  00000000  00000002  RWIX
  INT11                 0000ff96   00000002  00000000  00000002  RWIX
  INT12                 0000ff98   00000002  00000000  00000002  RWIX
  INT13                 0000ff9a   00000002  00000000  00000002  RWIX
  INT14                 0000ff9c   00000002  00000000  00000002  RWIX
  INT15                 0000ff9e   00000002  00000000  00000002  RWIX
  INT16                 0000ffa0   00000002  00000000  00000002  RWIX
  INT17                 0000ffa2   00000002  00000000  00000002  RWIX
  INT18                 0000ffa4   00000002  00000000  00000002  RWIX
  INT19                 0000ffa6   00000002  00000000  00000002  RWIX
  INT20                 0000ffa8   00000002  00000000  00000002  RWIX
  INT21                 0000ffaa   00000002  00000000  00000002  RWIX
  INT22                 0000ffac   00000002  00000000  00000002  RWIX
  INT23                 0000ffae   00000002  00000000  00000002  RWIX
  INT24                 0000ffb0   00000002  00000000  00000002  RWIX
  INT25                 0000ffb2   00000002  00000000  00000002  RWIX
  INT26                 0000ffb4   00000002  00000000  00000002  RWIX
  INT27                 0000ffb6   00000002  00000000  00000002  RWIX
  INT28                 0000ffb8   00000002  00000000  00000002  RWIX
  INT29                 0000ffba   00000002  00000000  00000002  RWIX
  INT30                 0000ffbc   00000002  00000000  00000002  RWIX
  INT31                 0000ffbe   00000002  00000000  00000002  RWIX
  INT32                 0000ffc0   00000002  00000000  00000002  RWIX
  INT33                 0000ffc2   00000002  00000000  00000002  RWIX
  INT34                 0000ffc4   00000002  00000000  00000002  RWIX
  INT35                 0000ffc6   00000002  00000000  00000002  RWIX
  INT36                 0000ffc8   00000002  00000000  00000002  RWIX
  INT37                 0000ffca   00000002  00000000  00000002  RWIX
  INT38                 0000ffcc   00000002  00000000  00000002  RWIX
  INT39                 0000ffce   00000002  00000000  00000002  RWIX
  INT40                 0000ffd0   00000002  00000000  00000002  RWIX
  INT41                 0000ffd2   00000002  00000002  00000000  RWIX
  INT42                 0000ffd4   00000002  00000002  00000000  RWIX
  INT43                 0000ffd6   00000002  00000002  00000000  RWIX
  INT44                 0000ffd8   00000002  00000002  00000000  RWIX
  INT45                 0000ffda   00000002  00000002  00000000  RWIX
  INT46                 0000ffdc   00000002  00000002  00000000  RWIX
  INT47                 0000ffde   00000002  00000002  00000000  RWIX
  INT48                 0000ffe0   00000002  00000002  00000000  RWIX
  INT49                 0000ffe2   00000002  00000002  00000000  RWIX
  INT50                 0000ffe4   00000002  00000002  00000000  RWIX
  INT51                 0000ffe6   00000002  00000002  00000000  RWIX
  INT52                 0000ffe8   00000002  00000002  00000000  RWIX
  INT53                 0000ffea   00000002  00000002  00000000  RWIX
  INT54                 0000ffec   00000002  00000002  00000000  RWIX
  INT55                 0000ffee   00000002  00000002  00000000  RWIX
  INT56                 0000fff0   00000002  00000002  00000000  RWIX
  INT57                 0000fff2   00000002  00000002  00000000  RWIX
  INT58                 0000fff4   00000002  00000002  00000000  RWIX
  INT59                 0000fff6   00000002  00000002  00000000  RWIX
  INT60                 0000fff8   00000002  00000002  00000000  RWIX
  INT61                 0000fffa   00000002  00000002  00000000  RWIX
  INT62                 0000fffc   00000002  00000002  00000000  RWIX
  RESET                 0000fffe   00000002  00000002  00000000  RWIX
  FLASH2                00010000   00014400  0000d7de  00006c22  RWIX


SECTION ALLOCATION MAP

 output                                  attributes/
section   page    origin      length       input sections
--------  ----  ----------  ----------   ----------------
.data      0    00002400    000005b8     UNINITIALIZED
                  00002400    000000c8     rts430x_lc_rd_eabi.lib : defs.obj (.data:_ftable)
                  000024c8    000000b0                            : signal.obj (.data:sigtable)
                  00002578    00000080                            : xvalues.obj (.data)
                  000025f8    00000078                            : lowlev.obj (.data:_device)
                  00002670    0000006c     console.obj (.data:ADS126xRegisterNames)
                  000026dc    00000064     console.obj (.data:outString)
                  00002740    00000064     main.obj (.data:wholeString)
                  000027a4    00000040     console.obj (.data:scr_mux_norm_strings)
                  000027e4    00000040     console.obj (.data:scr_speed_norm_strings)
                  00002824    0000003c     rts430x_lc_rd_eabi.lib : lowlev.obj (.data:_stream)
                  00002860    00000030     console.obj (.data:scr_idacdir_norm_strings)
                  00002890    0000002c     console.obj (.data:scr_idacmag_norm_strings)
                  000028bc    00000020     console.obj (.data:scr_gpio_norm_strings)
                  000028dc    00000020     console.obj (.data:scr_pga_norm_strings)
                  000028fc    00000019     console.obj (.data:tempString)
                  00002915    00000001     console.obj (.data)
                  00002916    00000014     console.obj (.data:scr_adc2ref_norm_strings)
                  0000292a    00000014     console.obj (.data:scr_filter_norm_strings)
                  0000293e    00000014     console.obj (.data:scr_refn_norm_strings)
                  00002952    00000014     console.obj (.data:scr_refp_norm_strings)
                  00002966    00000012     ac_bridge.obj (.data)
                  00002978    00000010     console.obj (.data:scr_adc2speed_norm_strings)
                  00002988    00000008     ucs.obj (.data)
                  00002990    00000008     rts430x_lc_rd_eabi.lib : feraiseexcept.obj (.data)
                  00002998    00000008     usb.obj (.data)
                  000029a0    00000004     rts430x_lc_rd_eabi.lib : exit_gvars.obj (.data:__TI_cleanup_ptr)
                  000029a4    00000004                            : exit_gvars.obj (.data:__TI_dtors_ptr)
                  000029a8    00000004                            : _lock.obj (.data:_lock)
                  000029ac    00000004                            : _lock.obj (.data:_unlock)
                  000029b0    00000002                            : defs.obj (.data)
                  000029b2    00000002                            : errno.obj (.data)
                  000029b4    00000002                            : memory.obj (.data)
                  000029b6    00000001     hal.obj (.data)
                  000029b7    00000001     main.obj (.data)

.sysmem    0    000029b8    00000190     UNINITIALIZED
                  000029b8    00000006     rts430x_lc_rd_eabi.lib : memory.obj (.sysmem)
                  000029be    0000018a     --HOLE--

.bss       0    00002b48    0000012c     UNINITIALIZED
                  00002b48    000000a0     (.common:__TI_tmpnams)
                  00002be8    00000022     (.common:abramSerialStringDescriptor)
                  00002c0a    0000001a     (.common:CdcReadCtrl)
                  00002c24    0000000c     (.common:CdcWriteCtrl)
                  00002c30    00000008     (.common:CdcControl)
                  00002c38    00000008     (.common:abUsbRequestIncomingData)
                  00002c40    00000008     (.common:abUsbRequestReturnData)
                  00002c48    00000008     (.common:parmbuf)
                  00002c50    00000004     (.common:USB_RX_memcpy)
                  00002c54    00000004     (.common:USB_TX_memcpy)
                  00002c58    00000004     (.common:pbIEP0Buffer)
                  00002c5c    00000004     (.common:pbOEP0Buffer)
                  00002c60    00000004     (.common:sys_base)
                  00002c64    00000004     (.common:sys_free)
                  00002c68    00000002     (.common:memsize)
                  00002c6a    00000002     (.common:wBytesRemainingOnIEP0)
                  00002c6c    00000002     (.common:wBytesRemainingOnOEP0)
                  00002c6e    00000002     (.common:wUsbEventMask)
                  00002c70    00000001     (.common:bConfigurationNumber)
                  00002c71    00000001     (.common:bInterfaceNumber)
                  00002c72    00000001     (.common:bRemoteWakeup)
                  00002c73    00000001     (.common:bStatusAction)

.cio       0    00002c74    00000120     UNINITIALIZED
                  00002c74    00000120     rts430x_lc_rd_eabi.lib : trgmsg.obj (.cio)

.stack     0    00004270    00000190     UNINITIALIZED
                  00004270    00000004     rts430x_lc_rd_eabi.lib : boot.obj (.stack)
                  00004274    0000018c     --HOLE--

.text:_isr 
*          0    00004400    0000024a     
                  00004400    000001b0     UsbIsr.obj (.text:_isr:iUsbInterruptHandler)
                  000045b0    0000004c     interrupts.obj (.text:_isr:UNMI_ISR)
                  000045fc    0000001e     interrupts.obj (.text:_isr:PORT1_ISR)
                  0000461a    0000001c     rts430x_lc_rd_eabi.lib : boot_special.obj (.text:_isr:_c_int00_noargs)
                  00004636    0000000e     interrupts.obj (.text:_isr:TIMER0_A0_ISR)
                  00004644    00000006     rts430x_lc_rd_eabi.lib : isr_trap.obj (.text:_isr:__TI_ISR_TRAP)

.const     0    0000464a    00005559     
                  0000464a    00002cc0     gpio.obj (.const:.string)
                  0000730a    00000a46     ucs.obj (.const:.string)
                  00007d50    00000920     console.obj (.const:.string)
                  00008670    000006fe     dma.obj (.const:.string)
                  00008d6e    000005e2     usci_b_spi.obj (.const:.string)
                  00009350    00000182     ac_bridge.obj (.const:.string)
                  000094d2    00000162     adc2_demo.obj (.const:.string)
                  00009634    00000156     ADS126x.obj (.const:.string)
                  0000978a    0000010a     descriptors.obj (.const:tUsbRequestList)
                  00009894    00000101     rts430x_lc_rd_eabi.lib : ctype.obj (.const:.string:_ctypes_)
                  00009995    00000001     adc2_demo.obj (.const)
                  00009996    000000a0     pmm.obj (.const:.string)
                  00009a36    00000096     descriptors.obj (.const:.string:abromStringDescriptor)
                  00009acc    00000043     descriptors.obj (.const)
                  00009b0f    00000001     --HOLE-- [fill = 0]
                  00009b10    00000026     rts430x_lc_rd_eabi.lib : _printfi.obj (.const:.string)
                  00009b36    00000020     usb.obj (.const:.string)
                  00009b56    00000018     rts430x_lc_rd_eabi.lib : xexp.obj (.const:s)
                  00009b6e    00000012     descriptors.obj (.const:.string:abromDeviceDescriptor)
                  00009b80    00000010     rts430x_lc_rd_eabi.lib : xexp.obj (.const:c)
                  00009b90    00000010     descriptors.obj (.const:stUsbHandle)
                  00009ba0    00000003     ac_bridge.obj (.const:.string:$P$T0$1)

.cinit     0    00009ba4    000002b6     
                  00009ba4    00000285     (.cinit..data.load) [load image, compression = rle]
                  00009e29    00000001     --HOLE-- [fill = 0]
                  00009e2a    0000000c     (__TI_handler_table)
                  00009e36    00000006     (.cinit..bss.load) [load image, compression = zero_init]
                  00009e3c    00000006     (.cinit..cio.load) [load image, compression = zero_init]
                  00009e42    00000018     (__TI_cinit_table)

.init_array 
*          0    00004400    00000000     UNINITIALIZED

.TI.persistent 
*          0    00002400    00000000     UNINITIALIZED

.TI.noinit 
*          0    00002b48    00000000     UNINITIALIZED

RTC        0    0000ffd2    00000002     
                  0000ffd2    00000002     rts430x_lc_rd_eabi.lib : int41.obj (.int41)

PORT2      0    0000ffd4    00000002     
                  0000ffd4    00000002     rts430x_lc_rd_eabi.lib : int42.obj (.int42)

TIMER2_A1 
*          0    0000ffd6    00000002     
                  0000ffd6    00000002     rts430x_lc_rd_eabi.lib : int43.obj (.int43)

TIMER2_A0 
*          0    0000ffd8    00000002     
                  0000ffd8    00000002     rts430x_lc_rd_eabi.lib : int44.obj (.int44)

USCI_B1    0    0000ffda    00000002     
                  0000ffda    00000002     rts430x_lc_rd_eabi.lib : int45.obj (.int45)

USCI_A1    0    0000ffdc    00000002     
                  0000ffdc    00000002     rts430x_lc_rd_eabi.lib : int46.obj (.int46)

PORT1      0    0000ffde    00000002     
                  0000ffde    00000002     interrupts.obj (.int47)

TIMER1_A1 
*          0    0000ffe0    00000002     
                  0000ffe0    00000002     rts430x_lc_rd_eabi.lib : int48.obj (.int48)

TIMER1_A0 
*          0    0000ffe2    00000002     
                  0000ffe2    00000002     rts430x_lc_rd_eabi.lib : int49.obj (.int49)

DMA        0    0000ffe4    00000002     
                  0000ffe4    00000002     rts430x_lc_rd_eabi.lib : int50.obj (.int50)

USB_UBM    0    0000ffe6    00000002     
                  0000ffe6    00000002     UsbIsr.obj (.int51)

TIMER0_A1 
*          0    0000ffe8    00000002     
                  0000ffe8    00000002     rts430x_lc_rd_eabi.lib : int52.obj (.int52)

TIMER0_A0 
*          0    0000ffea    00000002     
                  0000ffea    00000002     interrupts.obj (.int53)

ADC12      0    0000ffec    00000002     
                  0000ffec    00000002     rts430x_lc_rd_eabi.lib : int54.obj (.int54)

USCI_B0    0    0000ffee    00000002     
                  0000ffee    00000002     rts430x_lc_rd_eabi.lib : int55.obj (.int55)

USCI_A0    0    0000fff0    00000002     
                  0000fff0    00000002     rts430x_lc_rd_eabi.lib : int56.obj (.int56)

WDT        0    0000fff2    00000002     
                  0000fff2    00000002     rts430x_lc_rd_eabi.lib : int57.obj (.int57)

TIMER0_B1 
*          0    0000fff4    00000002     
                  0000fff4    00000002     rts430x_lc_rd_eabi.lib : int58.obj (.int58)

TIMER0_B0 
*          0    0000fff6    00000002     
                  0000fff6    00000002     rts430x_lc_rd_eabi.lib : int59.obj (.int59)

COMP_B     0    0000fff8    00000002     
                  0000fff8    00000002     rts430x_lc_rd_eabi.lib : int60.obj (.int60)

UNMI       0    0000fffa    00000002     
                  0000fffa    00000002     interrupts.obj (.int61)

SYSNMI     0    0000fffc    00000002     
                  0000fffc    00000002     rts430x_lc_rd_eabi.lib : int62.obj (.int62)

.reset     0    0000fffe    00000002     
                  0000fffe    00000002     rts430x_lc_rd_eabi.lib : boot.obj (.reset)

.text      0    00010000    0000d7de     
                  00010000    00000caa     console.obj (.text:show_parms)
                  00010caa    0000052c     UsbCdc.obj (.text:USBCDC_receiveData)
                  000111d6    00000476     ac_bridge.obj (.text:get_reference)
                  0001164c    00000452     rts430x_lc_rd_eabi.lib : frcdivd.obj (.text:__TI_frcdivd)
                  00011a9e    00000430     adc2_demo.obj (.text:ADS126xReadADC1SlowerThanADC2)
                  00011ece    000003fe     adc2_demo.obj (.text:ADS126xReadADC1FasterThanADC2)
                  000122cc    000003fc     adc2_demo.obj (.text:ADS126xReadADC1EqualToADC2)
                  000126c8    0000039a     rts430x_lc_rd_eabi.lib : div64u.obj (.text:__mspabi_divull)
                  00012a62    00000388                            : xexp.obj (.text:_Exp)
                  00012dea    0000033e     UsbCdc.obj (.text:CdcToHostFromBuffer)
                  00013128    00000326     ac_bridge.obj (.text:get_temperature)
                  0001344e    000002e4     rts430x_lc_rd_eabi.lib : frcmpyd.obj (.text:__TI_frcmpyd)
                  00013732    000002d8                            : addd.obj (.text:__mspabi_addd)
                  00013a0a    000002c6     console.obj (.text:set_gpio)
                  00013cd0    000002b4     console.obj (.text:console)
                  00013f84    000002a0     console.obj (.text:set_vref)
                  00014224    00000282     rts430x_lc_rd_eabi.lib : mpyd.obj (.text:__mspabi_mpyd)
                  000144a6    00000278     UsbCdc.obj (.text:CdcToBufferFromHost)
                  0001471e    00000262     rts430x_lc_rd_eabi.lib : _printfi.obj (.text:_setfield)
                  00014980    00000252                            : frcaddd.obj (.text:__TI_frcaddd)
                  00014bd2    00000222                            : divd.obj (.text:__mspabi_divd)
                  00014df4    00000218                            : _printfi.obj (.text:_pproc_fgea)
                  0001500c    00000218                            : _printfi.obj (.text:ecvt)
                  00015224    00000212                            : _printfi.obj (.text:acvt)
                  00015436    00000202                            : _printfi.obj (.text:__TI_printfi)
                  00015638    00000202                            : _printfi.obj (.text:fcvt)
                  0001583a    000001e6     gpio.obj (.text:GPIO_setAsInputPin)
                  00015a20    000001d8     usb.obj (.text:USB_reset)
                  00015bf8    000001d2     console.obj (.text:set_idac)
                  00015dca    000001cc     rts430x_lc_rd_eabi.lib : strtoul.obj (.text:strtoul)
                  00015f96    000001c8     console.obj (.text:retInString)
                  0001615e    000001c8     ac_bridge.obj (.text:run_ReadChopCont)
                  00016326    000001b6     gpio.obj (.text:GPIO_setAsOutputPin)
                  000164dc    000001b6     gpio.obj (.text:GPIO_setAsPeripheralModuleFunctionInputPin)
                  00016692    000001b6     gpio.obj (.text:GPIO_setAsPeripheralModuleFunctionOutputPin)
                  00016848    000001ae     ucs.obj (.text:privateUCSSourceClockFromDCO)
                  000169f6    000001a4     rts430x_lc_rd_eabi.lib : _printfi.obj (.text:_pconv_e)
                  00016b9a    0000019e                            : xdscale.obj (.text:_Dscale)
                  00016d38    0000019a     console.obj (.text:set_mux)
                  00016ed2    00000188     rts430x_lc_rd_eabi.lib : _printfi.obj (.text:_getarg_diouxp)
                  0001705a    00000186     gpio.obj (.text:GPIO_setOutputHighOnPin)
                  000171e0    00000186     gpio.obj (.text:GPIO_setOutputLowOnPin)
                  00017366    00000186     gpio.obj (.text:GPIO_toggleOutputOnPin)
                  000174ec    00000170     ucs.obj (.text:UCS_clockSignalInit)
                  0001765c    00000170     console.obj (.text:hex2asc)
                  000177cc    0000016e     rts430x_lc_rd_eabi.lib : _printfi.obj (.text:_pconv_a)
                  0001793a    00000152     ucs.obj (.text:privateUCSComputeCLKFrequency)
                  00017a8c    00000148     rts430x_lc_rd_eabi.lib : _printfi.obj (.text:_pproc_diouxp)
                  00017bd4    00000144     usb.obj (.text:USB_InitSerialStringDescriptor)
                  00017d18    00000136     UsbCdc.obj (.text:CopyUsbToBuff)
                  00017e4e    0000012e     ucs.obj (.text:UCS_initFLL)
                  00017f7c    00000126     dma.obj (.text:DMA_init)
                  000180a2    00000126     console.obj (.text:adc2_mux)
                  000181c8    00000126     hal.obj (.text:initPorts)
                  000182ee    00000120     UsbCdc.obj (.text:USBCDC_intfStatus)
                  0001840e    00000110     ac_bridge.obj (.text:set_excitation)
                  0001851e    00000108     pmm.obj (.text:PMM_setVCoreUp)
                  00018626    00000108     gpio.obj (.text:privateGPIOGetBaseAddress)
                  0001872e    00000106     ADS126x.obj (.text:ADS126xReadData)
                  00018834    00000100     rts430x_lc_rd_eabi.lib : xdnorm.obj (.text:_Dnorm)
                  00018934    000000fc     gpio.obj (.text:GPIO_interruptEdgeSelect)
                  00018a30    000000fc     rts430x_lc_rd_eabi.lib : _printfi.obj (.text:_pconv_g)
                  00018b2c    000000fa                            : _printfi.obj (.text:_pproc_fwp)
                  00018c26    000000fa     usb.obj (.text:usbDecodeAndProcessUsbRequest)
                  00018d20    000000f8     usb.obj (.text:USB_enable)
                  00018e18    000000f6     usci_b_spi.obj (.text:USCI_B_SPI_masterInit)
                  00018f0e    000000f0     UsbCdc.obj (.text:USBCDC_bytesInUSBBuffer)
                  00018ffe    000000f0     rts430x_lc_rd_eabi.lib : exp2.obj (.text:exp2)
                  000190ee    000000f0                            : fputs.obj (.text:fputs)
                  000191de    000000ee     console.obj (.text:set_datarate)
                  000192cc    000000ec     console.obj (.text:set_register)
                  000193b8    000000e0     rts430x_lc_rd_eabi.lib : setvbuf.obj (.text:setvbuf)
                  00019498    000000dc     console.obj (.text:set_chop)
                  00019574    000000dc     console.obj (.text:set_conv_mode)
                  00019650    000000d8     rts430x_lc_rd_eabi.lib : cmpd.obj (.text:__mspabi_cmpd)
                  00019728    000000d6     console.obj (.text:set_filter)
                  000197fe    000000d0     console.obj (.text:set_bias)
                  000198ce    000000ce     ac_bridge.obj (.text:run_ReadPosCont)
                  0001999c    000000cc     gpio.obj (.text:GPIO_clearInterruptFlag)
                  00019a68    000000cc     gpio.obj (.text:GPIO_disableInterrupt)
                  00019b34    000000cc     gpio.obj (.text:GPIO_enableInterrupt)
                  00019c00    000000c6     adc2_demo.obj (.text:LoadInitRegSettings)
                  00019cc6    000000c4     main.obj (.text:USBtask)
                  00019d8a    000000c2     UsbCdc.obj (.text:USBCDC_sendData)
                  00019e4c    000000c0     ac_bridge.obj (.text:LoadInitRegSettings)
                  00019f0c    000000c0     pmm.obj (.text:PMM_setVCoreDown)
                  00019fcc    000000be     ac_bridge.obj (.text:set_exc)
                  0001a08a    000000ba     usb.obj (.text:USB_determineFreq)
                  0001a144    000000ba     rts430x_lc_rd_eabi.lib : memory.obj (.text:malloc)
                  0001a1fe    000000b2                            : renormd.obj (.text:__TI_renormd)
                  0001a2b0    000000ae     ucs.obj (.text:UCS_LFXT1Start)
                  0001a35e    000000ae     usbConstructs.obj (.text:cdcSendDataWaitTilDone)
                  0001a40c    000000aa     usb.obj (.text:USB_init)
                  0001a4b6    000000aa     console.obj (.text:adc2_startstop)
                  0001a560    000000a8     rts430x_lc_rd_eabi.lib : _printfi.obj (.text:_pproc_str)
                  0001a608    000000a6     usbConstructs.obj (.text:cdcReceiveDataInBuffer)
                  0001a6ae    000000a6     usb.obj (.text:usbGetEndpointStatus)
                  0001a754    000000a4     console.obj (.text:set_pga)
                  0001a7f8    000000a2     usbConstructs.obj (.text:cdcSendDataInBackground)
                  0001a89a    000000a0     UsbCdc.obj (.text:usbGetLineCoding)
                  0001a93a    0000009e     rts430x_lc_rd_eabi.lib : trgdrv.obj (.text:HOSTlseek)
                  0001a9d8    0000009e                            : _printfi.obj (.text:_ltostr)
                  0001aa76    0000009a     pmm.obj (.text:PMM_setVCore)
                  0001ab10    00000098     ac_bridge.obj (.text:run_demo)
                  0001aba8    00000096     usb.obj (.text:USB_connectionState)
                  0001ac3e    00000096     console.obj (.text:adc2_datarate)
                  0001acd4    00000096     console.obj (.text:adc2_reference)
                  0001ad6a    00000094     rts430x_lc_rd_eabi.lib : fltlid.obj (.text:__mspabi_fltlid)
                  0001adfe    00000094                            : _printfi.obj (.text:_ecpy)
                  0001ae92    00000090     tlv.obj (.text:TLV_getInfo)
                  0001af22    00000090     rts430x_lc_rd_eabi.lib : _printfi.obj (.text:_mcpy)
                  0001afb2    0000008e                            : memory.obj (.text:free)
                  0001b040    0000008c     console.obj (.text:adc2_pga)
                  0001b0cc    00000088     rts430x_lc_rd_eabi.lib : _printfi.obj (.text:_div)
                  0001b154    00000086                            : ldexp.obj (.text:ldexp)
                  0001b1da    00000082     dma.obj (.text:DMA_setDstAddress)
                  0001b25c    00000082     UsbIsr.obj (.text:PWRVBUSoffHandler)
                  0001b2de    00000080     rts430x_lc_rd_eabi.lib : ltoa.obj (.text:ltoa)
                  0001b35e    00000080     usb.obj (.text:usbSendNextPacketOnIEP0)
                  0001b3de    0000007e     dma.obj (.text:DMA_setSrcAddress)
                  0001b45c    0000007e     rts430x_lc_rd_eabi.lib : _io_perm.obj (.text:__TI_wrt_ok)
                  0001b4da    0000007a     usbdma.obj (.text:memcpyDMA)
                  0001b554    0000007a     ac_bridge.obj (.text:show_AppMenu)
                  0001b5ce    00000078     UsbCdc.obj (.text:Handler_SetLineCoding)
                  0001b646    00000078     rts430x_lc_rd_eabi.lib : _printfi.obj (.text:_pconv_f)
                  0001b6be    00000078     usb.obj (.text:usbGetStringDescriptor)
                  0001b736    00000076     rts430x_lc_rd_eabi.lib : fltuld.obj (.text:__mspabi_fltuld)
                  0001b7ac    00000074                            : trgdrv.obj (.text:HOSTrename)
                  0001b820    00000072                            : xdunscal.obj (.text:_Dunscale)
                  0001b892    00000070     UsbIsr.obj (.text:PWRVBUSonHandler)
                  0001b902    00000070     rts430x_lc_rd_eabi.lib : fclose.obj (.text:__TI_closefile)
                  0001b972    0000006e                            : trgdrv.obj (.text:HOSTopen)
                  0001b9e0    0000006c                            : autoinit_wdt.obj (.text:_auto_init_hold_wdt)
                  0001ba4c    0000006c     console.obj (.text:adc2)
                  0001bab8    0000006a     rts430x_lc_rd_eabi.lib : trgdrv.obj (.text:HOSTwrite)
                  0001bb22    0000006a     ucs.obj (.text:UCS_XT2StartWithTimeout)
                  0001bb8c    0000006a     rts430x_lc_rd_eabi.lib : fseek.obj (.text:fseek)
                  0001bbf6    0000006a     usb.obj (.text:usbReceiveNextPacketOnOEP0)
                  0001bc60    00000068     rts430x_lc_rd_eabi.lib : trgdrv.obj (.text:HOSTread)
                  0001bcc8    00000068                            : copy_decompress_rle.obj (.text:__TI_decompress_rle_core)
                  0001bd30    00000066     ADS126x.obj (.text:ADS126xReadRegister)
                  0001bd96    00000066     rts430x_lc_rd_eabi.lib : fixdli.obj (.text:__mspabi_fixdli)
                  0001bdfc    00000066     adc2_demo.obj (.text:show_AppMenu)
                  0001be62    00000064     rts430x_lc_rd_eabi.lib : fflush.obj (.text:__TI_doflush)
                  0001bec6    00000064     hal.obj (.text:initClocks)
                  0001bf2a    00000062     ADS126x.obj (.text:ADS126xWriteRegister)
                  0001bf8c    00000062     rts430x_lc_rd_eabi.lib : atoi.obj (.text:atoi)
                  0001bfee    00000062                            : snprintf.obj (.text:snprintf)
                  0001c050    0000005c     UsbIsr.obj (.text:SetupPacketInterruptHandler)
                  0001c0ac    0000005a     rts430x_lc_rd_eabi.lib : lowlev.obj (.text:close)
                  0001c106    0000005a                            : lowlev.obj (.text:getdevice)
                  0001c160    0000005a     adc2_demo.obj (.text:run_adc2_demo)
                  0001c1ba    00000058     rts430x_lc_rd_eabi.lib : fflush.obj (.text:fflush)
                  0001c212    00000058     usbdma.obj (.text:memcpyV)
                  0001c26a    00000058     rts430x_lc_rd_eabi.lib : div32u.obj (.text)
                  0001c2c2    00000056     usb.obj (.text:usbSetEndpointFeature)
                  0001c318    00000054     hal.obj (.text:initSPI)
                  0001c36c    00000054     usb.obj (.text:usbClearEndpointFeature)
                  0001c3c0    00000050     rts430x_lc_rd_eabi.lib : xdclass.obj (.text:_Dclass)
                  0001c410    0000004e     ucs.obj (.text:UCS_initFLLSettle)
                  0001c45e    0000004e     rts430x_lc_rd_eabi.lib : _printfi.obj (.text:_fcpy)
                  0001c4ac    0000004c                            : trgdrv.obj (.text:HOSTclose)
                  0001c4f8    0000004a     UsbCdc.obj (.text:CdcResetData)
                  0001c542    0000004a     usb.obj (.text:USB_setup)
                  0001c58c    00000048     console.obj (.text:print2Console)
                  0001c5d4    00000046     rts430x_lc_rd_eabi.lib : trgdrv.obj (.text:HOSTunlink)
                  0001c61a    00000046                            : _printfi.obj (.text:_pproc_fflags)
                  0001c660    00000044                            : sprintf.obj (.text:sprintf)
                  0001c6a4    00000042                            : frexp.obj (.text:frexp)
                  0001c6e6    00000042                            : memory.obj (.text:minit)
                  0001c728    00000040     console.obj (.text:PressANYkeytoContinue)
                  0001c768    00000040     usb.obj (.text:USB_connectionInfo)
                  0001c7a8    00000040     usbdma.obj (.text:USB_initMemcpy)
                  0001c7e8    00000040     rts430x_lc_rd_eabi.lib : div32s.obj (.text)
                  0001c828    0000003e                            : _printfi.obj (.text:incr_hex)
                  0001c866    0000003e                            : asr32.obj (.text:l_asr_const)
                  0001c8a4    0000003e                            : lsl32.obj (.text:l_lsl_const)
                  0001c8e2    0000003e                            : lsr32.obj (.text:l_lsr_const)
                  0001c920    0000003e                            : lowlev.obj (.text:lseek)
                  0001c95e    0000003c     ADS126x.obj (.text:ADS126xXferByte)
                  0001c99a    0000003c     UsbIsr.obj (.text:OEP0InterruptHandler)
                  0001c9d6    0000003c     ucs.obj (.text:UCS_XT2Start)
                  0001ca12    0000003c     rts430x_lc_rd_eabi.lib : lowlev.obj (.text:write)
                  0001ca4e    0000003a     usci_b_spi.obj (.text:USCI_B_SPI_disableInterrupt)
                  0001ca88    0000003a     rts430x_lc_rd_eabi.lib : lsl64.obj (.text:__mspabi_sllll)
                  0001cac2    0000003a                            : lsr64.obj (.text:__mspabi_srlll)
                  0001cafc    0000003a     console.obj (.text:show_version)
                  0001cb36    00000038     ADS126x.obj (.text:set_adc_CS)
                  0001cb6e    00000038     ADS126x.obj (.text:set_adc_START)
                  0001cba6    00000038     rts430x_lc_rd_eabi.lib : signal.obj (.text:signal)
                  0001cbde    00000038     usb.obj (.text:usbSendDataPacketOnEP0)
                  0001cc16    00000036     rts430x_lc_rd_eabi.lib : xferaise.obj (.text:_Feraise)
                  0001cc4c    00000036                            : fopen.obj (.text:__TI_cleanup)
                  0001cc82    00000036                            : trgmsg.obj (.text:__TI_writemsg)
                  0001ccb8    00000036                            : snprintf.obj (.text:_outs)
                  0001ccee    00000034     wdt_a.obj (.text:WDT_A_hold)
                  0001cd22    00000034     rts430x_lc_rd_eabi.lib : feraiseexcept.obj (.text:feraiseexcept)
                  0001cd56    00000034     usb.obj (.text:usbDisableInEndpointInterrupt)
                  0001cd8a    00000034     usb.obj (.text:usbDisableOutEndpointInterrupt)
                  0001cdbe    00000032     ucs.obj (.text:UCS_getSMCLK)
                  0001cdf0    00000032     rts430x_lc_rd_eabi.lib : trgmsg.obj (.text:__TI_readmsg)
                  0001ce22    00000032                            : subd.obj (.text:__mspabi_subd)
                  0001ce54    00000032     main.obj (.text:main)
                  0001ce86    00000032     rts430x_lc_rd_eabi.lib : raise.obj (.text:raise)
                  0001ceb8    00000032                            : strncpy.obj (.text:strncpy)
                  0001ceea    00000032     usb.obj (.text:usbGetDeviceStatus)
                  0001cf1c    00000032     usb.obj (.text:usbSetConfiguration)
                  0001cf4e    00000030     dma.obj (.text:DMA_disableTransfers)
                  0001cf7e    00000030     dma.obj (.text:DMA_enableTransfers)
                  0001cfae    00000030     ucs.obj (.text:UCS_setExternalClockSource)
                  0001cfde    00000030     usb.obj (.text:USB_suspend)
                  0001d00e    00000030     rts430x_lc_rd_eabi.lib : lowlev.obj (.text:unlink)
                  0001d03e    0000002e     dma.obj (.text:DMA_startTransfer)
                  0001d06c    0000002e     rts430x_lc_rd_eabi.lib : negd.obj (.text:__mspabi_negd)
                  0001d09a    0000002e                            : exit.obj (.text:exit)
                  0001d0c8    0000002e                            : lowlev.obj (.text:finddevice)
                  0001d0f6    0000002c     dma.obj (.text:DMA_getInterruptStatus)
                  0001d122    0000002c     rts430x_lc_rd_eabi.lib : div16s.obj (.text)
                  0001d14e    00000028     hal.obj (.text:WaitForDRDY)
                  0001d176    00000028     rts430x_lc_rd_eabi.lib : fixdi.obj (.text:__mspabi_fixdi)
                  0001d19e    00000026     ucs.obj (.text:UCS_clearFaultFlag)
                  0001d1c4    00000024     rts430x_lc_rd_eabi.lib : copy_zero_init.obj (.text:decompress:ZI:__TI_zero_init)
                  0001d1e8    00000024     usb.obj (.text:usbReceiveDataPacketOnEP0)
                  0001d20c    00000022     UsbCdc.obj (.text:CdcIsReceiveInProgress)
                  0001d22e    00000022     usb.obj (.text:USB_disable)
                  0001d250    00000022     usci_b_spi.obj (.text:USCI_B_SPI_transmitData)
                  0001d272    00000022     rts430x_lc_rd_eabi.lib : mult32_f5hw.obj (.text)
                  0001d294    00000020                            : snprintf.obj (.text:_outc)
                  0001d2b4    00000020                            : sprintf.obj (.text:_outs)
                  0001d2d4    00000020     usb.obj (.text:usbSetAddress)
                  0001d2f4    00000020     rts430x_lc_rd_eabi.lib : _printfi.obj (.text:val_hex)
                  0001d314    0000001e     dma.obj (.text:DMA_setTransferSize)
                  0001d332    0000001e     rts430x_lc_rd_eabi.lib : memccpy.obj (.text:memccpy)
                  0001d350    0000001e                            : strcat.obj (.text:strcat)
                  0001d36e    0000001e     usb.obj (.text:usbGetInterface)
                  0001d38c    0000001e     usb.obj (.text:usbGetInterfaceStatus)
                  0001d3aa    0000001c     UsbIsr.obj (.text:IEP0InterruptHandler)
                  0001d3c6    0000001c     usci_b_spi.obj (.text:USCI_B_SPI_isBusy)
                  0001d3e2    0000001c     rts430x_lc_rd_eabi.lib : strchr.obj (.text:strchr)
                  0001d3fe    0000001c                            : strcmp.obj (.text:strcmp)
                  0001d41a    0000001a     usb.obj (.text:USB_connect)
                  0001d434    0000001a     usci_b_spi.obj (.text:USCI_B_SPI_receiveData)
                  0001d44e    0000001a     rts430x_lc_rd_eabi.lib : assert.obj (.text:_abort_msg)
                  0001d468    00000018     usbEventHandling.obj (.text:USBCDC_handleSetLineCoding)
                  0001d480    00000018     usb.obj (.text:USB_resume)
                  0001d498    00000018     usci_b_spi.obj (.text:USCI_B_SPI_enable)
                  0001d4b0    00000018     usb.obj (.text:usbClearDeviceFeature)
                  0001d4c8    00000018     usb.obj (.text:usbSetDeviceFeature)
                  0001d4e0    00000016     ADS126x.obj (.text:ADS126xSendADC2StartCommand)
                  0001d4f6    00000016     ADS126x.obj (.text:ADS126xSendADC2StopCommand)
                  0001d50c    00000016     rts430x_lc_rd_eabi.lib : memchr.obj (.text:memchr)
                  0001d522    00000016                            : memset.obj (.text:memset)
                  0001d538    00000016     console.obj (.text:printCommandPrompt)
                  0001d54e    00000016     console.obj (.text:printError)
                  0001d564    00000016     rts430x_lc_rd_eabi.lib : div16u.obj (.text)
                  0001d57a    00000016                            : mult16_f5hw.obj (.text)
                  0001d590    00000016     usb.obj (.text:usbGetConfigurationDescriptor)
                  0001d5a6    00000016     usb.obj (.text:usbGetDeviceDescriptor)
                  0001d5bc    00000014     usbEventHandling.obj (.text:USB_handleVbusOnEvent)
                  0001d5d0    00000014     rts430x_lc_rd_eabi.lib : sprintf.obj (.text:_outc)
                  0001d5e4    00000014                            : memcpy.obj (.text:memcpy)
                  0001d5f8    00000014     usb.obj (.text:usbGetConfiguration)
                  0001d60c    00000014     UsbCdc.obj (.text:usbSetControlLineState)
                  0001d620    00000012     rts430x_lc_rd_eabi.lib : copy_decompress_none.obj (.text:decompress:none:__TI_decompress_none)
                  0001d632    00000012                            : strcpy.obj (.text:strcpy)
                  0001d644    00000012                            : tolower.obj (.text:tolower)
                  0001d656    00000012                            : toupper.obj (.text:toupper)
                  0001d668    00000012     usb.obj (.text:usbSetInterface)
                  0001d67a    00000010     usbEventHandling.obj (.text:USBCDC_handleDataReceived)
                  0001d68a    00000010     usbEventHandling.obj (.text:USBCDC_handleSetControlLineState)
                  0001d69a    00000010     usb.obj (.text:USB_setEnabledEvents)
                  0001d6aa    00000010     rts430x_lc_rd_eabi.lib : asr32.obj (.text:l_asr)
                  0001d6ba    00000010                            : lsl32.obj (.text:l_lsl)
                  0001d6ca    00000010                            : lsr32.obj (.text:l_lsr)
                  0001d6da    0000000e     sfr.obj (.text:SFR_clearInterrupt)
                  0001d6e8    0000000e     rts430x_lc_rd_eabi.lib : strlen.obj (.text:strlen)
                  0001d6f6    0000000e     usb.obj (.text:usbInvalidRequest)
                  0001d704    0000000e     usb.obj (.text:usbRestoreInEndpointInterrupt)
                  0001d712    0000000e     usb.obj (.text:usbRestoreOutEndpointInterrupt)
                  0001d720    0000000e     usb.obj (.text:usbSendZeroLengthPacketOnIEP0)
                  0001d72e    0000000c     usbEventHandling.obj (.text:USBCDC_handleReceiveCompleted)
                  0001d73a    0000000c     usbEventHandling.obj (.text:USBCDC_handleSendCompleted)
                  0001d746    0000000c     rts430x_lc_rd_eabi.lib : fltid.obj (.text:__mspabi_fltid)
                  0001d752    0000000c     UsbCdc.obj (.text:usbSetLineCoding)
                  0001d75e    0000000a     rts430x_lc_rd_eabi.lib : abs.obj (.text:abs)
                  0001d768    0000000a                            : lsl16.obj (.text)
                  0001d772    0000000a                            : lsr16.obj (.text)
                  0001d77c    0000000a     usb.obj (.text:usbStallEndpoint0)
                  0001d786    00000008     ucs.obj (.text:UCS_XT2Off)
                  0001d78e    00000008     usbEventHandling.obj (.text:USB_handleVbusOffEvent)
                  0001d796    00000006     dma.obj (.text:DMA_disableTransferDuringReadModifyWrite)
                  0001d79c    00000006     dma.obj (.text:DMA_enableTransferDuringReadModifyWrite)
                  0001d7a2    00000006     usb.obj (.text:USB_getVersion)
                  0001d7a8    00000006     rts430x_lc_rd_eabi.lib : fltud.obj (.text:__mspabi_fltud)
                  0001d7ae    00000006                            : copy_decompress_rle.obj (.text:decompress:rle24:__TI_decompress_rle24)
                  0001d7b4    00000006     usb.obj (.text:usbClearOEP0ByteCount)
                  0001d7ba    00000006     usb.obj (.text:usbStallOEP0)
                  0001d7c0    00000004     usbEventHandling.obj (.text:USB_handleClockEvent)
                  0001d7c4    00000004     usbEventHandling.obj (.text:USB_handleEnumCompleteEvent)
                  0001d7c8    00000004     usbEventHandling.obj (.text:USB_handleResetEvent)
                  0001d7cc    00000004     usbEventHandling.obj (.text:USB_handleResumeEvent)
                  0001d7d0    00000004     usbEventHandling.obj (.text:USB_handleSuspendEvent)
                  0001d7d4    00000004     rts430x_lc_rd_eabi.lib : pre_init.obj (.text:_system_pre_init)
                  0001d7d8    00000004                            : exit.obj (.text:abort)
                  0001d7dc    00000002                            : _lock.obj (.text:_nop)


LINKER GENERATED COPY TABLES

__TI_cinit_table @ 00009e42 records: 3, size/record: 8, table size: 24
	.data: load addr=00009ba4, load size=00000285 bytes, run addr=00002400, run size=000005b8 bytes, compression=rle
	.bss: load addr=00009e36, load size=00000006 bytes, run addr=00002b48, run size=0000012c bytes, compression=zero_init
	.cio: load addr=00009e3c, load size=00000006 bytes, run addr=00002c74, run size=00000120 bytes, compression=zero_init


LINKER GENERATED HANDLER TABLE

__TI_handler_table @ 00009e2a records: 3, size/record: 4, table size: 12
	index: 0, handler: __TI_zero_init
	index: 1, handler: __TI_decompress_rle24
	index: 2, handler: __TI_decompress_none


GLOBAL SYMBOLS: SORTED ALPHABETICALLY BY Name 

address   name                                       
-------   ----                                       
00000700  ADC12CTL0                                  
00000701  ADC12CTL0_H                                
00000700  ADC12CTL0_L                                
00000702  ADC12CTL1                                  
00000703  ADC12CTL1_H                                
00000702  ADC12CTL1_L                                
00000704  ADC12CTL2                                  
00000705  ADC12CTL2_H                                
00000704  ADC12CTL2_L                                
0000070c  ADC12IE                                    
0000070d  ADC12IE_H                                  
0000070c  ADC12IE_L                                  
0000070a  ADC12IFG                                   
0000070b  ADC12IFG_H                                 
0000070a  ADC12IFG_L                                 
0000070e  ADC12IV                                    
0000070f  ADC12IV_H                                  
0000070e  ADC12IV_L                                  
00000710  ADC12MCTL0                                 
00000711  ADC12MCTL1                                 
0000071a  ADC12MCTL10                                
0000071b  ADC12MCTL11                                
0000071c  ADC12MCTL12                                
0000071d  ADC12MCTL13                                
0000071e  ADC12MCTL14                                
0000071f  ADC12MCTL15                                
00000712  ADC12MCTL2                                 
00000713  ADC12MCTL3                                 
00000714  ADC12MCTL4                                 
00000715  ADC12MCTL5                                 
00000716  ADC12MCTL6                                 
00000717  ADC12MCTL7                                 
00000718  ADC12MCTL8                                 
00000719  ADC12MCTL9                                 
00000720  ADC12MEM0                                  
00000721  ADC12MEM0_H                                
00000720  ADC12MEM0_L                                
00000722  ADC12MEM1                                  
00000734  ADC12MEM10                                 
00000735  ADC12MEM10_H                               
00000734  ADC12MEM10_L                               
00000736  ADC12MEM11                                 
00000737  ADC12MEM11_H                               
00000736  ADC12MEM11_L                               
00000738  ADC12MEM12                                 
00000739  ADC12MEM12_H                               
00000738  ADC12MEM12_L                               
0000073a  ADC12MEM13                                 
0000073b  ADC12MEM13_H                               
0000073a  ADC12MEM13_L                               
0000073c  ADC12MEM14                                 
0000073d  ADC12MEM14_H                               
0000073c  ADC12MEM14_L                               
0000073e  ADC12MEM15                                 
0000073f  ADC12MEM15_H                               
0000073e  ADC12MEM15_L                               
00000723  ADC12MEM1_H                                
00000722  ADC12MEM1_L                                
00000724  ADC12MEM2                                  
00000725  ADC12MEM2_H                                
00000724  ADC12MEM2_L                                
00000726  ADC12MEM3                                  
00000727  ADC12MEM3_H                                
00000726  ADC12MEM3_L                                
00000728  ADC12MEM4                                  
00000729  ADC12MEM4_H                                
00000728  ADC12MEM4_L                                
0000072a  ADC12MEM5                                  
0000072b  ADC12MEM5_H                                
0000072a  ADC12MEM5_L                                
0000072c  ADC12MEM6                                  
0000072d  ADC12MEM6_H                                
0000072c  ADC12MEM6_L                                
0000072e  ADC12MEM7                                  
0000072f  ADC12MEM7_H                                
0000072e  ADC12MEM7_L                                
00000730  ADC12MEM8                                  
00000731  ADC12MEM8_H                                
00000730  ADC12MEM8_L                                
00000732  ADC12MEM9                                  
00000733  ADC12MEM9_H                                
00000732  ADC12MEM9_L                                
0001872e  ADS126xReadData                            
0001bd30  ADS126xReadRegister                        
00002670  ADS126xRegisterNames                       
0001d4e0  ADS126xSendADC2StartCommand                
0001d4f6  ADS126xSendADC2StopCommand                 
0001bf2a  ADS126xWriteRegister                       
0001c95e  ADS126xXferByte                            
0001d7d8  C$$EXIT                                    
0001ccb4  C$$IO$$                                    
000008c0  CBCTL0                                     
000008c1  CBCTL0_H                                   
000008c0  CBCTL0_L                                   
000008c2  CBCTL1                                     
000008c3  CBCTL1_H                                   
000008c2  CBCTL1_L                                   
000008c4  CBCTL2                                     
000008c5  CBCTL2_H                                   
000008c4  CBCTL2_L                                   
000008c6  CBCTL3                                     
000008c7  CBCTL3_H                                   
000008c6  CBCTL3_L                                   
000008cc  CBINT                                      
000008cd  CBINT_H                                    
000008cc  CBINT_L                                    
000008ce  CBIV                                       
00000150  CRCDI                                      
00000152  CRCDIRB                                    
00000153  CRCDIRB_H                                  
00000152  CRCDIRB_L                                  
00000151  CRCDI_H                                    
00000150  CRCDI_L                                    
00000154  CRCINIRES                                  
00000155  CRCINIRES_H                                
00000154  CRCINIRES_L                                
00000156  CRCRESR                                    
00000157  CRCRESR_H                                  
00000156  CRCRESR_L                                  
0001d20c  CdcIsReceiveInProgress                     
0001c4f8  CdcResetData                               
000144a6  CdcToBufferFromHost                        
00012dea  CdcToHostFromBuffer                        
00017d18  CopyUsbToBuff                              
00000510  DMA0CTL                                    
00000511  DMA0CTL_H                                  
00000510  DMA0CTL_L                                  
00000516  DMA0DA                                     
00000518  DMA0DAH                                    
00000516  DMA0DAL                                    
00000512  DMA0SA                                     
00000514  DMA0SAH                                    
00000512  DMA0SAL                                    
0000051a  DMA0SZ                                     
00000520  DMA1CTL                                    
00000521  DMA1CTL_H                                  
00000520  DMA1CTL_L                                  
00000526  DMA1DA                                     
00000528  DMA1DAH                                    
00000526  DMA1DAL                                    
00000522  DMA1SA                                     
00000524  DMA1SAH                                    
00000522  DMA1SAL                                    
0000052a  DMA1SZ                                     
00000530  DMA2CTL                                    
00000531  DMA2CTL_H                                  
00000530  DMA2CTL_L                                  
00000536  DMA2DA                                     
00000538  DMA2DAH                                    
00000536  DMA2DAL                                    
00000532  DMA2SA                                     
00000534  DMA2SAH                                    
00000532  DMA2SAL                                    
0000053a  DMA2SZ                                     
00000500  DMACTL0                                    
00000501  DMACTL0_H                                  
00000500  DMACTL0_L                                  
00000502  DMACTL1                                    
00000503  DMACTL1_H                                  
00000502  DMACTL1_L                                  
00000504  DMACTL2                                    
00000505  DMACTL2_H                                  
00000504  DMACTL2_L                                  
00000506  DMACTL3                                    
00000507  DMACTL3_H                                  
00000506  DMACTL3_L                                  
00000508  DMACTL4                                    
00000509  DMACTL4_H                                  
00000508  DMACTL4_L                                  
0000050e  DMAIV                                      
0000050f  DMAIV_H                                    
0000050e  DMAIV_L                                    
0001d796  DMA_disableTransferDuringReadModifyWrite   
0001cf4e  DMA_disableTransfers                       
0001d79c  DMA_enableTransferDuringReadModifyWrite    
0001cf7e  DMA_enableTransfers                        
0001d0f6  DMA_getInterruptStatus                     
00017f7c  DMA_init                                   
0001b1da  DMA_setDstAddress                          
0001b3de  DMA_setSrcAddress                          
0001d314  DMA_setTransferSize                        
0001d03e  DMA_startTransfer                          
00000140  FCTL1                                      
00000141  FCTL1_H                                    
00000140  FCTL1_L                                    
00000144  FCTL3                                      
00000145  FCTL3_H                                    
00000144  FCTL3_L                                    
00000146  FCTL4                                      
00000147  FCTL4_H                                    
00000146  FCTL4_L                                    
0001999c  GPIO_clearInterruptFlag                    
00019a68  GPIO_disableInterrupt                      
00019b34  GPIO_enableInterrupt                       
00018934  GPIO_interruptEdgeSelect                   
0001583a  GPIO_setAsInputPin                         
00016326  GPIO_setAsOutputPin                        
000164dc  GPIO_setAsPeripheralModuleFunctionInputPin 
00016692  GPIO_setAsPeripheralModuleFunctionOutputPin
0001705a  GPIO_setOutputHighOnPin                    
000171e0  GPIO_setOutputLowOnPin                     
00017366  GPIO_toggleOutputOnPin                     
0001c4ac  HOSTclose                                  
0001a93a  HOSTlseek                                  
0001b972  HOSTopen                                   
0001bc60  HOSTread                                   
0001b7ac  HOSTrename                                 
0001c5d4  HOSTunlink                                 
0001bab8  HOSTwrite                                  
0001b5ce  Handler_SetLineCoding                      
0001d3aa  IEP0InterruptHandler                       
000004c4  MAC                                        
000004da  MAC32H                                     
000004db  MAC32H_H                                   
000004da  MAC32H_L                                   
000004d8  MAC32L                                     
000004d9  MAC32L_H                                   
000004d8  MAC32L_L                                   
000004c6  MACS                                       
000004de  MACS32H                                    
000004df  MACS32H_H                                  
000004de  MACS32H_L                                  
000004dc  MACS32L                                    
000004dd  MACS32L_H                                  
000004dc  MACS32L_L                                  
000004c7  MACS_H                                     
000004c6  MACS_L                                     
000004c5  MAC_H                                      
000004c4  MAC_L                                      
000004c0  MPY                                        
000004ec  MPY32CTL0                                  
000004ed  MPY32CTL0_H                                
000004ec  MPY32CTL0_L                                
000004d2  MPY32H                                     
000004d3  MPY32H_H                                   
000004d2  MPY32H_L                                   
000004d0  MPY32L                                     
000004d1  MPY32L_H                                   
000004d0  MPY32L_L                                   
000004c2  MPYS                                       
000004d6  MPYS32H                                    
000004d7  MPYS32H_H                                  
000004d6  MPYS32H_L                                  
000004d4  MPYS32L                                    
000004d5  MPYS32L_H                                  
000004d4  MPYS32L_L                                  
000004c3  MPYS_H                                     
000004c2  MPYS_L                                     
000004c1  MPY_H                                      
000004c0  MPY_L                                      
00009995  MinNumADCReadings                          
0001c99a  OEP0InterruptHandler                       
000004c8  OP2                                        
000004e2  OP2H                                       
000004e3  OP2H_H                                     
000004e2  OP2H_L                                     
000004e0  OP2L                                       
000004e1  OP2L_H                                     
000004e0  OP2L_L                                     
000004c9  OP2_H                                      
000004c8  OP2_L                                      
0000020e  P1IV                                       
0000021e  P2IV                                       
000001e0  P4MAP01                                    
000001e1  P4MAP01_H                                  
000001e0  P4MAP01_L                                  
000001e2  P4MAP23                                    
000001e3  P4MAP23_H                                  
000001e2  P4MAP23_L                                  
000001e4  P4MAP45                                    
000001e5  P4MAP45_H                                  
000001e4  P4MAP45_L                                  
000001e6  P4MAP67                                    
000001e7  P4MAP67_H                                  
000001e6  P4MAP67_L                                  
00000204  PADIR                                      
00000205  PADIR_H                                    
00000204  PADIR_L                                    
00000208  PADS                                       
00000209  PADS_H                                     
00000208  PADS_L                                     
0000021a  PAIE                                       
00000218  PAIES                                      
00000219  PAIES_H                                    
00000218  PAIES_L                                    
0000021b  PAIE_H                                     
0000021a  PAIE_L                                     
0000021c  PAIFG                                      
0000021d  PAIFG_H                                    
0000021c  PAIFG_L                                    
00000200  PAIN                                       
00000201  PAIN_H                                     
00000200  PAIN_L                                     
00000202  PAOUT                                      
00000203  PAOUT_H                                    
00000202  PAOUT_L                                    
00000206  PAREN                                      
00000207  PAREN_H                                    
00000206  PAREN_L                                    
0000020a  PASEL                                      
0000020b  PASEL_H                                    
0000020a  PASEL_L                                    
00000224  PBDIR                                      
00000225  PBDIR_H                                    
00000224  PBDIR_L                                    
00000228  PBDS                                       
00000229  PBDS_H                                     
00000228  PBDS_L                                     
00000220  PBIN                                       
00000221  PBIN_H                                     
00000220  PBIN_L                                     
00000222  PBOUT                                      
00000223  PBOUT_H                                    
00000222  PBOUT_L                                    
00000226  PBREN                                      
00000227  PBREN_H                                    
00000226  PBREN_L                                    
0000022a  PBSEL                                      
0000022b  PBSEL_H                                    
0000022a  PBSEL_L                                    
00000244  PCDIR                                      
00000245  PCDIR_H                                    
00000244  PCDIR_L                                    
00000248  PCDS                                       
00000249  PCDS_H                                     
00000248  PCDS_L                                     
00000240  PCIN                                       
00000241  PCIN_H                                     
00000240  PCIN_L                                     
00000242  PCOUT                                      
00000243  PCOUT_H                                    
00000242  PCOUT_L                                    
00000246  PCREN                                      
00000247  PCREN_H                                    
00000246  PCREN_L                                    
0000024a  PCSEL                                      
0000024b  PCSEL_H                                    
0000024a  PCSEL_L                                    
00000264  PDDIR                                      
00000265  PDDIR_H                                    
00000264  PDDIR_L                                    
00000268  PDDS                                       
00000269  PDDS_H                                     
00000268  PDDS_L                                     
00000260  PDIN                                       
00000261  PDIN_H                                     
00000260  PDIN_L                                     
00000262  PDOUT                                      
00000263  PDOUT_H                                    
00000262  PDOUT_L                                    
00000266  PDREN                                      
00000267  PDREN_H                                    
00000266  PDREN_L                                    
0000026a  PDSEL                                      
0000026b  PDSEL_H                                    
0000026a  PDSEL_L                                    
00000324  PJDIR                                      
00000325  PJDIR_H                                    
00000324  PJDIR_L                                    
00000328  PJDS                                       
00000329  PJDS_H                                     
00000328  PJDS_L                                     
00000320  PJIN                                       
00000321  PJIN_H                                     
00000320  PJIN_L                                     
00000322  PJOUT                                      
00000323  PJOUT_H                                    
00000322  PJOUT_L                                    
00000326  PJREN                                      
00000327  PJREN_H                                    
00000326  PJREN_L                                    
00000130  PM5CTL0                                    
00000131  PM5CTL0_H                                  
00000130  PM5CTL0_L                                  
000001c2  PMAPCTL                                    
000001c3  PMAPCTL_H                                  
000001c2  PMAPCTL_L                                  
000001c0  PMAPKEYID                                  
000001c1  PMAPKEYID_H                                
000001c0  PMAPKEYID_L                                
00000120  PMMCTL0                                    
00000121  PMMCTL0_H                                  
00000120  PMMCTL0_L                                  
00000122  PMMCTL1                                    
00000123  PMMCTL1_H                                  
00000122  PMMCTL1_L                                  
0000012c  PMMIFG                                     
0000012d  PMMIFG_H                                   
0000012c  PMMIFG_L                                   
0000012e  PMMRIE                                     
0000012f  PMMRIE_H                                   
0000012e  PMMRIE_L                                   
0001aa76  PMM_setVCore                               
00019f0c  PMM_setVCoreDown                           
0001851e  PMM_setVCoreUp                             
000045fc  PORT1_ISR                                  
0001b25c  PWRVBUSoffHandler                          
0001b892  PWRVBUSonHandler                           
0001c728  PressANYkeytoContinue                      
00000158  RCCTL0                                     
00000159  RCCTL0_H                                   
00000158  RCCTL0_L                                   
000001b0  REFCTL0                                    
000001b1  REFCTL0_H                                  
000001b0  REFCTL0_L                                  
000004e4  RES0                                       
000004e5  RES0_H                                     
000004e4  RES0_L                                     
000004e6  RES1                                       
000004e7  RES1_H                                     
000004e6  RES1_L                                     
000004e8  RES2                                       
000004e9  RES2_H                                     
000004e8  RES2_L                                     
000004ea  RES3                                       
000004eb  RES3_H                                     
000004ea  RES3_L                                     
000004cc  RESHI                                      
000004cd  RESHI_H                                    
000004cc  RESHI_L                                    
000004ca  RESLO                                      
000004cb  RESLO_H                                    
000004ca  RESLO_L                                    
000004ba  RTCADOWDAY                                 
000004bb  RTCADOWDAY_H                               
000004ba  RTCADOWDAY_L                               
000004b8  RTCAMINHR                                  
000004b9  RTCAMINHR_H                                
000004b8  RTCAMINHR_L                                
000004a0  RTCCTL01                                   
000004a1  RTCCTL01_H                                 
000004a0  RTCCTL01_L                                 
000004a2  RTCCTL23                                   
000004a3  RTCCTL23_H                                 
000004a2  RTCCTL23_L                                 
000004b4  RTCDATE                                    
000004b5  RTCDATE_H                                  
000004b4  RTCDATE_L                                  
000004ae  RTCIV                                      
000004ac  RTCPS                                      
000004a8  RTCPS0CTL                                  
000004a9  RTCPS0CTL_H                                
000004a8  RTCPS0CTL_L                                
000004aa  RTCPS1CTL                                  
000004ab  RTCPS1CTL_H                                
000004aa  RTCPS1CTL_L                                
000004ad  RTCPS_H                                    
000004ac  RTCPS_L                                    
000004b0  RTCTIM0                                    
000004b1  RTCTIM0_H                                  
000004b0  RTCTIM0_L                                  
000004b2  RTCTIM1                                    
000004b3  RTCTIM1_H                                  
000004b2  RTCTIM1_L                                  
000004b6  RTCYEAR                                    
000004b7  RTCYEAR_H                                  
000004b6  RTCYEAR_L                                  
00000100  SFRIE1                                     
00000101  SFRIE1_H                                   
00000100  SFRIE1_L                                   
00000102  SFRIFG1                                    
00000103  SFRIFG1_H                                  
00000102  SFRIFG1_L                                  
00000104  SFRRPCR                                    
00000105  SFRRPCR_H                                  
00000104  SFRRPCR_L                                  
0001d6da  SFR_clearInterrupt                         
000004ce  SUMEXT                                     
000004cf  SUMEXT_H                                   
000004ce  SUMEXT_L                                   
00000124  SVSMHCTL                                   
00000125  SVSMHCTL_H                                 
00000124  SVSMHCTL_L                                 
00000128  SVSMIO                                     
00000129  SVSMIO_H                                   
00000128  SVSMIO_L                                   
00000126  SVSMLCTL                                   
00000127  SVSMLCTL_H                                 
00000126  SVSMLCTL_L                                 
00000198  SYSBERRIV                                  
00000199  SYSBERRIV_H                                
00000198  SYSBERRIV_L                                
00000182  SYSBSLC                                    
00000183  SYSBSLC_H                                  
00000182  SYSBSLC_L                                  
00000180  SYSCTL                                     
00000181  SYSCTL_H                                   
00000180  SYSCTL_L                                   
00000186  SYSJMBC                                    
00000187  SYSJMBC_H                                  
00000186  SYSJMBC_L                                  
00000188  SYSJMBI0                                   
00000189  SYSJMBI0_H                                 
00000188  SYSJMBI0_L                                 
0000018a  SYSJMBI1                                   
0000018b  SYSJMBI1_H                                 
0000018a  SYSJMBI1_L                                 
0000018c  SYSJMBO0                                   
0000018d  SYSJMBO0_H                                 
0000018c  SYSJMBO0_L                                 
0000018e  SYSJMBO1                                   
0000018f  SYSJMBO1_H                                 
0000018e  SYSJMBO1_L                                 
0000019e  SYSRSTIV                                   
0000019f  SYSRSTIV_H                                 
0000019e  SYSRSTIV_L                                 
0000019c  SYSSNIV                                    
0000019d  SYSSNIV_H                                  
0000019c  SYSSNIV_L                                  
0000019a  SYSUNIV                                    
0000019b  SYSUNIV_H                                  
0000019a  SYSUNIV_L                                  
0001c050  SetupPacketInterruptHandler                
00000352  TA0CCR0                                    
00000354  TA0CCR1                                    
00000356  TA0CCR2                                    
00000358  TA0CCR3                                    
0000035a  TA0CCR4                                    
00000342  TA0CCTL0                                   
00000344  TA0CCTL1                                   
00000346  TA0CCTL2                                   
00000348  TA0CCTL3                                   
0000034a  TA0CCTL4                                   
00000340  TA0CTL                                     
00000360  TA0EX0                                     
0000036e  TA0IV                                      
00000350  TA0R                                       
00000392  TA1CCR0                                    
00000394  TA1CCR1                                    
00000396  TA1CCR2                                    
00000382  TA1CCTL0                                   
00000384  TA1CCTL1                                   
00000386  TA1CCTL2                                   
00000380  TA1CTL                                     
000003a0  TA1EX0                                     
000003ae  TA1IV                                      
00000390  TA1R                                       
00000412  TA2CCR0                                    
00000414  TA2CCR1                                    
00000416  TA2CCR2                                    
00000402  TA2CCTL0                                   
00000404  TA2CCTL1                                   
00000406  TA2CCTL2                                   
00000400  TA2CTL                                     
00000420  TA2EX0                                     
0000042e  TA2IV                                      
00000410  TA2R                                       
000003d2  TB0CCR0                                    
000003d4  TB0CCR1                                    
000003d6  TB0CCR2                                    
000003d8  TB0CCR3                                    
000003da  TB0CCR4                                    
000003dc  TB0CCR5                                    
000003de  TB0CCR6                                    
000003c2  TB0CCTL0                                   
000003c4  TB0CCTL1                                   
000003c6  TB0CCTL2                                   
000003c8  TB0CCTL3                                   
000003ca  TB0CCTL4                                   
000003cc  TB0CCTL5                                   
000003ce  TB0CCTL6                                   
000003c0  TB0CTL                                     
000003e0  TB0EX0                                     
000003ee  TB0IV                                      
000003d0  TB0R                                       
00004636  TIMER0_A0_ISR                              
0001ae92  TLV_getInfo                                
000005d0  UCA0ABCTL                                  
000005c6  UCA0BRW                                    
000005c7  UCA0BRW_H                                  
000005c6  UCA0BRW_L                                  
000005c0  UCA0CTLW0                                  
000005c1  UCA0CTLW0_H                                
000005c0  UCA0CTLW0_L                                
000005dc  UCA0ICTL                                   
000005dd  UCA0ICTL_H                                 
000005dc  UCA0ICTL_L                                 
000005d2  UCA0IRCTL                                  
000005d3  UCA0IRCTL_H                                
000005d2  UCA0IRCTL_L                                
000005de  UCA0IV                                     
000005c8  UCA0MCTL                                   
000005cc  UCA0RXBUF                                  
000005ca  UCA0STAT                                   
000005ce  UCA0TXBUF                                  
00000610  UCA1ABCTL                                  
00000606  UCA1BRW                                    
00000607  UCA1BRW_H                                  
00000606  UCA1BRW_L                                  
00000600  UCA1CTLW0                                  
00000601  UCA1CTLW0_H                                
00000600  UCA1CTLW0_L                                
0000061c  UCA1ICTL                                   
0000061d  UCA1ICTL_H                                 
0000061c  UCA1ICTL_L                                 
00000612  UCA1IRCTL                                  
00000613  UCA1IRCTL_H                                
00000612  UCA1IRCTL_L                                
0000061e  UCA1IV                                     
00000608  UCA1MCTL                                   
0000060c  UCA1RXBUF                                  
0000060a  UCA1STAT                                   
0000060e  UCA1TXBUF                                  
000005e6  UCB0BRW                                    
000005e7  UCB0BRW_H                                  
000005e6  UCB0BRW_L                                  
000005e0  UCB0CTLW0                                  
000005e1  UCB0CTLW0_H                                
000005e0  UCB0CTLW0_L                                
000005f0  UCB0I2COA                                  
000005f1  UCB0I2COA_H                                
000005f0  UCB0I2COA_L                                
000005f2  UCB0I2CSA                                  
000005f3  UCB0I2CSA_H                                
000005f2  UCB0I2CSA_L                                
000005fc  UCB0ICTL                                   
000005fd  UCB0ICTL_H                                 
000005fc  UCB0ICTL_L                                 
000005fe  UCB0IV                                     
000005ec  UCB0RXBUF                                  
000005ea  UCB0STAT                                   
000005ee  UCB0TXBUF                                  
00000626  UCB1BRW                                    
00000627  UCB1BRW_H                                  
00000626  UCB1BRW_L                                  
00000620  UCB1CTLW0                                  
00000621  UCB1CTLW0_H                                
00000620  UCB1CTLW0_L                                
00000630  UCB1I2COA                                  
00000631  UCB1I2COA_H                                
00000630  UCB1I2COA_L                                
00000632  UCB1I2CSA                                  
00000633  UCB1I2CSA_H                                
00000632  UCB1I2CSA_L                                
0000063c  UCB1ICTL                                   
0000063d  UCB1ICTL_H                                 
0000063c  UCB1ICTL_L                                 
0000063e  UCB1IV                                     
0000062c  UCB1RXBUF                                  
0000062a  UCB1STAT                                   
0000062e  UCB1TXBUF                                  
00000160  UCSCTL0                                    
00000161  UCSCTL0_H                                  
00000160  UCSCTL0_L                                  
00000162  UCSCTL1                                    
00000163  UCSCTL1_H                                  
00000162  UCSCTL1_L                                  
00000164  UCSCTL2                                    
00000165  UCSCTL2_H                                  
00000164  UCSCTL2_L                                  
00000166  UCSCTL3                                    
00000167  UCSCTL3_H                                  
00000166  UCSCTL3_L                                  
00000168  UCSCTL4                                    
00000169  UCSCTL4_H                                  
00000168  UCSCTL4_L                                  
0000016a  UCSCTL5                                    
0000016b  UCSCTL5_H                                  
0000016a  UCSCTL5_L                                  
0000016c  UCSCTL6                                    
0000016d  UCSCTL6_H                                  
0000016c  UCSCTL6_L                                  
0000016e  UCSCTL7                                    
0000016f  UCSCTL7_H                                  
0000016e  UCSCTL7_L                                  
00000170  UCSCTL8                                    
00000171  UCSCTL8_H                                  
00000170  UCSCTL8_L                                  
0001a2b0  UCS_LFXT1Start                             
00002988  UCS_XT1ClockFrequency                      
0000298c  UCS_XT2ClockFrequency                      
0001d786  UCS_XT2Off                                 
0001c9d6  UCS_XT2Start                               
0001bb22  UCS_XT2StartWithTimeout                    
0001d19e  UCS_clearFaultFlag                         
000174ec  UCS_clockSignalInit                        
0001cdbe  UCS_getSMCLK                               
00017e4e  UCS_initFLL                                
0001c410  UCS_initFLLSettle                          
0001cfae  UCS_setExternalClockSource                 
000045b0  UNMI_ISR                                   
00018f0e  USBCDC_bytesInUSBBuffer                    
0001d67a  USBCDC_handleDataReceived                  
0001d72e  USBCDC_handleReceiveCompleted              
0001d73a  USBCDC_handleSendCompleted                 
0001d68a  USBCDC_handleSetControlLineState           
0001d468  USBCDC_handleSetLineCoding                 
000182ee  USBCDC_intfStatus                          
00010caa  USBCDC_receiveData                         
00019d8a  USBCDC_sendData                            
00000902  USBCNF                                     
00000903  USBCNF_H                                   
00000902  USBCNF_L                                   
0000093c  USBCTL                                     
0000093a  USBFN                                      
0000093b  USBFN_H                                    
0000093a  USBFN_L                                    
0000093f  USBFUNADR                                  
0000093d  USBIE                                      
00002378  USBIEP0BUF                                 
000023c9  USBIEPBBAX_1                               
000023d1  USBIEPBBAX_2                               
000023d9  USBIEPBBAX_3                               
000023e1  USBIEPBBAX_4                               
000023e9  USBIEPBBAX_5                               
000023f1  USBIEPBBAX_6                               
000023f9  USBIEPBBAX_7                               
000023cd  USBIEPBBAY_1                               
000023d5  USBIEPBBAY_2                               
000023dd  USBIEPBBAY_3                               
000023e5  USBIEPBBAY_4                               
000023ed  USBIEPBBAY_5                               
000023f5  USBIEPBBAY_6                               
000023fd  USBIEPBBAY_7                               
000023ca  USBIEPBCTX_1                               
000023d2  USBIEPBCTX_2                               
000023da  USBIEPBCTX_3                               
000023e2  USBIEPBCTX_4                               
000023ea  USBIEPBCTX_5                               
000023f2  USBIEPBCTX_6                               
000023fa  USBIEPBCTX_7                               
000023ce  USBIEPBCTY_1                               
000023d6  USBIEPBCTY_2                               
000023de  USBIEPBCTY_3                               
000023e6  USBIEPBCTY_4                               
000023ee  USBIEPBCTY_5                               
000023f6  USBIEPBCTY_6                               
000023fe  USBIEPBCTY_7                               
00000920  USBIEPCNF_0                                
000023c8  USBIEPCNF_1                                
000023d0  USBIEPCNF_2                                
000023d8  USBIEPCNF_3                                
000023e0  USBIEPCNF_4                                
000023e8  USBIEPCNF_5                                
000023f0  USBIEPCNF_6                                
000023f8  USBIEPCNF_7                                
00000921  USBIEPCNT_0                                
0000092e  USBIEPIE                                   
00000930  USBIEPIFG                                  
000023cf  USBIEPSIZXY_1                              
000023d7  USBIEPSIZXY_2                              
000023df  USBIEPSIZXY_3                              
000023e7  USBIEPSIZXY_4                              
000023ef  USBIEPSIZXY_5                              
000023f7  USBIEPSIZXY_6                              
000023ff  USBIEPSIZXY_7                              
0000093e  USBIFG                                     
00000900  USBKEYID                                   
00000901  USBKEYID_H                                 
00000900  USBKEYID_L                                 
00000936  USBMAINT                                   
00000937  USBMAINT_H                                 
00000936  USBMAINT_L                                 
00002370  USBOEP0BUF                                 
00002389  USBOEPBBAX_1                               
00002391  USBOEPBBAX_2                               
00002399  USBOEPBBAX_3                               
000023a1  USBOEPBBAX_4                               
000023a9  USBOEPBBAX_5                               
000023b1  USBOEPBBAX_6                               
000023b9  USBOEPBBAX_7                               
0000238d  USBOEPBBAY_1                               
00002395  USBOEPBBAY_2                               
0000239d  USBOEPBBAY_3                               
000023a5  USBOEPBBAY_4                               
000023ad  USBOEPBBAY_5                               
000023b5  USBOEPBBAY_6                               
000023bd  USBOEPBBAY_7                               
0000238a  USBOEPBCTX_1                               
00002392  USBOEPBCTX_2                               
0000239a  USBOEPBCTX_3                               
000023a2  USBOEPBCTX_4                               
000023aa  USBOEPBCTX_5                               
000023b2  USBOEPBCTX_6                               
000023ba  USBOEPBCTX_7                               
0000238e  USBOEPBCTY_1                               
00002396  USBOEPBCTY_2                               
0000239e  USBOEPBCTY_3                               
000023a6  USBOEPBCTY_4                               
000023ae  USBOEPBCTY_5                               
000023b6  USBOEPBCTY_6                               
000023be  USBOEPBCTY_7                               
00000922  USBOEPCNF_0                                
00002388  USBOEPCNF_1                                
00002390  USBOEPCNF_2                                
00002398  USBOEPCNF_3                                
000023a0  USBOEPCNF_4                                
000023a8  USBOEPCNF_5                                
000023b0  USBOEPCNF_6                                
000023b8  USBOEPCNF_7                                
00000923  USBOEPCNT_0                                
0000092f  USBOEPIE                                   
00000931  USBOEPIFG                                  
0000238f  USBOEPSIZXY_1                              
00002397  USBOEPSIZXY_2                              
0000239f  USBOEPSIZXY_3                              
000023a7  USBOEPSIZXY_4                              
000023af  USBOEPSIZXY_5                              
000023b7  USBOEPSIZXY_6                              
000023bf  USBOEPSIZXY_7                              
00000904  USBPHYCTL                                  
00000905  USBPHYCTL_H                                
00000904  USBPHYCTL_L                                
00000910  USBPLLCTL                                  
00000911  USBPLLCTL_H                                
00000910  USBPLLCTL_L                                
00000912  USBPLLDIVB                                 
00000913  USBPLLDIVB_H                               
00000912  USBPLLDIVB_L                               
00000914  USBPLLIR                                   
00000915  USBPLLIR_H                                 
00000914  USBPLLIR_L                                 
00000908  USBPWRCTL                                  
00000909  USBPWRCTL_H                                
00000908  USBPWRCTL_L                                
00001c00  USBSTABUFF                                 
00002380  USBSUBLK                                   
0000236f  USBTOPBUFF                                 
00000938  USBTSREG                                   
00000939  USBTSREG_H                                 
00000938  USBTSREG_L                                 
00000932  USBVECINT                                  
00000933  USBVECINT_H                                
00000932  USBVECINT_L                                
00017bd4  USB_InitSerialStringDescriptor             
00002c50  USB_RX_memcpy                              
00002c54  USB_TX_memcpy                              
0001d41a  USB_connect                                
0001c768  USB_connectionInfo                         
0001aba8  USB_connectionState                        
0001a08a  USB_determineFreq                          
0001d22e  USB_disable                                
00018d20  USB_enable                                 
0001d7a2  USB_getVersion                             
0001d7c0  USB_handleClockEvent                       
0001d7c4  USB_handleEnumCompleteEvent                
0001d7c8  USB_handleResetEvent                       
0001d7cc  USB_handleResumeEvent                      
0001d7d0  USB_handleSuspendEvent                     
0001d78e  USB_handleVbusOffEvent                     
0001d5bc  USB_handleVbusOnEvent                      
0001a40c  USB_init                                   
0001c7a8  USB_initMemcpy                             
00015a20  USB_reset                                  
0001d480  USB_resume                                 
0001d69a  USB_setEnabledEvents                       
0001c542  USB_setup                                  
0001cfde  USB_suspend                                
00019cc6  USBtask                                    
0001ca4e  USCI_B_SPI_disableInterrupt                
0001d498  USCI_B_SPI_enable                          
0001d3c6  USCI_B_SPI_isBusy                          
00018e18  USCI_B_SPI_masterInit                      
0001d434  USCI_B_SPI_receiveData                     
0001d250  USCI_B_SPI_transmitData                    
0000299c  VERSION                                    
0000015c  WDTCTL                                     
0000015d  WDTCTL_H                                   
0000015c  WDTCTL_L                                   
0001ccee  WDT_A_hold                                 
0001d14e  WaitForDRDY                                
00002c74  _CIOBUF_                                   
0001c3c0  _Dclass                                    
00002578  _Denorm                                    
00018834  _Dnorm                                     
00016b9a  _Dscale                                    
0001b820  _Dunscale                                  
00002588  _Eps                                       
000029b2  _Errno                                     
00012a62  _Exp                                       
00002990  _Fenv                                      
0001cc16  _Feraise                                   
00002598  _Hugeval                                   
000025a8  _Inf                                       
000025b8  _Nan                                       
000025d8  _Rteps                                     
000025c8  _Snan                                      
00002994  _Tls_setup__Fenv                           
000025e8  _Xbig                                      
000025f0  _Zero                                      
00004400  __STACK_END                                
00000190  __STACK_SIZE                               
00000190  __SYSMEM_SIZE                              
00009e42  __TI_CINIT_Base                            
00009e5a  __TI_CINIT_Limit                           
00009e2a  __TI_Handler_Table_Base                    
00009e36  __TI_Handler_Table_Limit                   
UNDEFED   __TI_INITARRAY_Base                        
UNDEFED   __TI_INITARRAY_Limit                       
00004644  __TI_ISR_TRAP                              
0001cc4c  __TI_cleanup                               
000029a0  __TI_cleanup_ptr                           
0001b902  __TI_closefile                             
0001d620  __TI_decompress_none                       
0001d7ae  __TI_decompress_rle24                      
0001be62  __TI_doflush                               
000029a4  __TI_dtors_ptr                             
00014980  __TI_frcaddd                               
0001164c  __TI_frcdivd                               
0001344e  __TI_frcmpyd                               
000029b0  __TI_ft_end                                
0000ffd2  __TI_int41                                 
0000ffd4  __TI_int42                                 
0000ffd6  __TI_int43                                 
0000ffd8  __TI_int44                                 
0000ffda  __TI_int45                                 
0000ffdc  __TI_int46                                 
0000ffde  __TI_int47                                 
0000ffe0  __TI_int48                                 
0000ffe2  __TI_int49                                 
0000ffe4  __TI_int50                                 
0000ffe6  __TI_int51                                 
0000ffe8  __TI_int52                                 
0000ffea  __TI_int53                                 
0000ffec  __TI_int54                                 
0000ffee  __TI_int55                                 
0000fff0  __TI_int56                                 
0000fff2  __TI_int57                                 
0000fff4  __TI_int58                                 
0000fff6  __TI_int59                                 
0000fff8  __TI_int60                                 
0000fffa  __TI_int61                                 
0000fffc  __TI_int62                                 
00015436  __TI_printfi                               
0001cdf0  __TI_readmsg                               
0001a1fe  __TI_renormd                               
00002b48  __TI_tmpnams                               
0001cc82  __TI_writemsg                              
0001b45c  __TI_wrt_ok                                
0001d1c4  __TI_zero_init                             
ffffffff  __binit__                                  
ffffffff  __c_args__                                 
00013732  __mspabi_addd                              
00019650  __mspabi_cmpd                              
00014bd2  __mspabi_divd                              
0001d122  __mspabi_divi                              
0001c7e8  __mspabi_divli                             
0001d564  __mspabi_divu                              
0001c26a  __mspabi_divul                             
000126c8  __mspabi_divull                            
0001d176  __mspabi_fixdi                             
0001bd96  __mspabi_fixdli                            
0001d746  __mspabi_fltid                             
0001ad6a  __mspabi_fltlid                            
0001d7a8  __mspabi_fltud                             
0001b736  __mspabi_fltuld                            
00014224  __mspabi_mpyd                              
0001d57a  __mspabi_mpyi_f5hw                         
0001d272  __mspabi_mpyl_f5hw                         
0001d06c  __mspabi_negd                              
0001d122  __mspabi_remi                              
0001c7e8  __mspabi_remli                             
0001d564  __mspabi_remu                              
0001c26a  __mspabi_remul                             
0001d768  __mspabi_slli                              
0001d6ba  __mspabi_slll                              
0001c8dc  __mspabi_slll_1                            
0001c8b8  __mspabi_slll_10                           
0001c8b4  __mspabi_slll_11                           
0001c8b0  __mspabi_slll_12                           
0001c8ac  __mspabi_slll_13                           
0001c8a8  __mspabi_slll_14                           
0001c8a4  __mspabi_slll_15                           
0001c8d8  __mspabi_slll_2                            
0001c8d4  __mspabi_slll_3                            
0001c8d0  __mspabi_slll_4                            
0001c8cc  __mspabi_slll_5                            
0001c8c8  __mspabi_slll_6                            
0001c8c4  __mspabi_slll_7                            
0001c8c0  __mspabi_slll_8                            
0001c8bc  __mspabi_slll_9                            
0001ca88  __mspabi_sllll                             
0001d6aa  __mspabi_sral                              
0001c89e  __mspabi_sral_1                            
0001c87a  __mspabi_sral_10                           
0001c876  __mspabi_sral_11                           
0001c872  __mspabi_sral_12                           
0001c86e  __mspabi_sral_13                           
0001c86a  __mspabi_sral_14                           
0001c866  __mspabi_sral_15                           
0001c89a  __mspabi_sral_2                            
0001c896  __mspabi_sral_3                            
0001c892  __mspabi_sral_4                            
0001c88e  __mspabi_sral_5                            
0001c88a  __mspabi_sral_6                            
0001c886  __mspabi_sral_7                            
0001c882  __mspabi_sral_8                            
0001c87e  __mspabi_sral_9                            
0001d772  __mspabi_srli                              
0001d6ca  __mspabi_srll                              
0001c91a  __mspabi_srll_1                            
0001c8f6  __mspabi_srll_10                           
0001c8f2  __mspabi_srll_11                           
0001c8ee  __mspabi_srll_12                           
0001c8ea  __mspabi_srll_13                           
0001c8e6  __mspabi_srll_14                           
0001c8e2  __mspabi_srll_15                           
0001c916  __mspabi_srll_2                            
0001c912  __mspabi_srll_3                            
0001c90e  __mspabi_srll_4                            
0001c90a  __mspabi_srll_5                            
0001c906  __mspabi_srll_6                            
0001c902  __mspabi_srll_7                            
0001c8fe  __mspabi_srll_8                            
0001c8fa  __mspabi_srll_9                            
0001cac2  __mspabi_srlll                             
0001ce22  __mspabi_subd                              
0001d44e  _abort_msg                                 
0001b9e0  _auto_init_hold_wdt                        
0000461a  _c_int00_noargs                            
00009894  _ctypes_                                   
00002400  _ftable                                    
000029a8  _lock                                      
0001d7dc  _nop                                       
0000fffe  _reset_vector                              
00004270  _stack                                     
000029b8  _sys_memory                                
0001d7d4  _system_pre_init                           
000029ac  _unlock                                    
00002378  abIEP0Buffer                               
00002370  abOEP0Buffer                               
00002c38  abUsbRequestIncomingData                   
00002c40  abUsbRequestReturnData                     
0001d7d8  abort                                      
00002be8  abramSerialStringDescriptor                
00009acc  abromConfigurationDescriptorGroup          
00009b6e  abromDeviceDescriptor                      
00009a36  abromStringDescriptor                      
0001d75e  abs                                        
0001ba4c  adc2                                       
0001ac3e  adc2_datarate                              
000180a2  adc2_mux                                   
0001b040  adc2_pga                                   
0001acd4  adc2_reference                             
0001a4b6  adc2_startstop                             
0001bf8c  atoi                                       
0000299a  bEnumerationStatus                         
00002999  bFunctionSuspended                         
00002c73  bStatusAction                              
ffffffff  binit                                      
0001a608  cdcReceiveDataInBuffer                     
0001a7f8  cdcSendDataInBackground                    
0001a35e  cdcSendDataWaitTilDone                     
0001c0ac  close                                      
00013cd0  console                                    
0001d09a  exit                                       
00018ffe  exp2                                       
0001cd22  feraiseexcept                              
0001c1ba  fflush                                     
000190ee  fputs                                      
0001afb2  free                                       
0001c6a4  frexp                                      
0001bb8c  fseek                                      
000029b6  g_DRDY_flag                                
000029b7  g_bCDCDataReceived_event                   
0001765c  hex2asc                                    
00004400  iUsbInterruptHandler                       
0001bec6  initClocks                                 
000181c8  initPorts                                  
0001c318  initSPI                                    
0001b154  ldexp                                      
0001c920  lseek                                      
0001b2de  ltoa                                       
0001ce54  main                                       
0001a144  malloc                                     
0001d332  memccpy                                    
0001d50c  memchr                                     
0001d5e4  memcpy                                     
0001b4da  memcpyDMA                                  
0001c212  memcpyV                                    
0001d522  memset                                     
0001c6e6  minit                                      
000026dc  outString                                  
00001c00  pbXBufferAddressEp1                        
00001d00  pbXBufferAddressEp2                        
00001e00  pbXBufferAddressEp3                        
00001f00  pbXBufferAddressEp4                        
00002000  pbXBufferAddressEp5                        
00002100  pbXBufferAddressEp6                        
00002200  pbXBufferAddressEp7                        
00001c80  pbXBufferAddressEp81                       
00001d80  pbXBufferAddressEp82                       
00001e80  pbXBufferAddressEp83                       
00001f80  pbXBufferAddressEp84                       
00002080  pbXBufferAddressEp85                       
00002180  pbXBufferAddressEp86                       
00002280  pbXBufferAddressEp87                       
00001c40  pbYBufferAddressEp1                        
00001d40  pbYBufferAddressEp2                        
00001e40  pbYBufferAddressEp3                        
00001f40  pbYBufferAddressEp4                        
00002040  pbYBufferAddressEp5                        
00002140  pbYBufferAddressEp6                        
00002240  pbYBufferAddressEp7                        
00001cc0  pbYBufferAddressEp81                       
00001dc0  pbYBufferAddressEp82                       
00001ec0  pbYBufferAddressEp83                       
00001fc0  pbYBufferAddressEp84                       
000020c0  pbYBufferAddressEp85                       
000021c0  pbYBufferAddressEp86                       
000022c0  pbYBufferAddressEp87                       
0001c58c  print2Console                              
0001d538  printCommandPrompt                         
0001d54e  printError                                 
0001ce86  raise                                      
0001d00e  remove                                     
00015f96  retInString                                
0001c160  run_adc2_demo                              
0001ab10  run_demo                                   
00002916  scr_adc2ref_norm_strings                   
00002978  scr_adc2speed_norm_strings                 
0000292a  scr_filter_norm_strings                    
000028bc  scr_gpio_norm_strings                      
00002860  scr_idacdir_norm_strings                   
00002890  scr_idacmag_norm_strings                   
000027a4  scr_mux_norm_strings                       
000028dc  scr_pga_norm_strings                       
0000293e  scr_refn_norm_strings                      
00002952  scr_refp_norm_strings                      
000027e4  scr_speed_norm_strings                     
0001cb36  set_adc_CS                                 
0001cb6e  set_adc_START                              
000197fe  set_bias                                   
00019498  set_chop                                   
00019574  set_conv_mode                              
000191de  set_datarate                               
00019fcc  set_exc                                    
00019728  set_filter                                 
00013a0a  set_gpio                                   
00015bf8  set_idac                                   
00016d38  set_mux                                    
0001a754  set_pga                                    
000192cc  set_register                               
00013f84  set_vref                                   
000193b8  setvbuf                                    
00010000  show_parms                                 
0001cafc  show_version                               
0001cba6  signal                                     
0001bfee  snprintf                                   
0001c660  sprintf                                    
00009b90  stUsbHandle                                
0001d350  strcat                                     
0001d3e2  strchr                                     
0001d3fe  strcmp                                     
0001d632  strcpy                                     
0001d6e8  strlen                                     
0001ceb8  strncpy                                    
00015dca  strtoul                                    
00000920  tEndPoint0DescriptorBlock                  
000023c8  tInputEndPointDescriptorBlock              
00002388  tOutputEndPointDescriptorBlock             
00002380  tSetupPacket                               
0000978a  tUsbRequestList                            
000028fc  tempString                                 
0001d644  tolower                                    
0001d656  toupper                                    
0001d00e  unlink                                     
0001d4b0  usbClearDeviceFeature                      
0001c36c  usbClearEndpointFeature                    
0001d7b4  usbClearOEP0ByteCount                      
00018c26  usbDecodeAndProcessUsbRequest              
0001cd56  usbDisableInEndpointInterrupt              
0001cd8a  usbDisableOutEndpointInterrupt             
0001d5f8  usbGetConfiguration                        
0001d590  usbGetConfigurationDescriptor              
0001d5a6  usbGetDeviceDescriptor                     
0001ceea  usbGetDeviceStatus                         
0001a6ae  usbGetEndpointStatus                       
0001d36e  usbGetInterface                            
0001d38c  usbGetInterfaceStatus                      
0001a89a  usbGetLineCoding                           
0001b6be  usbGetStringDescriptor                     
0001d6f6  usbInvalidRequest                          
0001d1e8  usbReceiveDataPacketOnEP0                  
0001bbf6  usbReceiveNextPacketOnOEP0                 
0001d704  usbRestoreInEndpointInterrupt              
0001d712  usbRestoreOutEndpointInterrupt             
0001cbde  usbSendDataPacketOnEP0                     
0001b35e  usbSendNextPacketOnIEP0                    
0001d720  usbSendZeroLengthPacketOnIEP0              
0001d2d4  usbSetAddress                              
0001cf1c  usbSetConfiguration                        
0001d60c  usbSetControlLineState                     
0001d4c8  usbSetDeviceFeature                        
0001c2c2  usbSetEndpointFeature                      
0001d668  usbSetInterface                            
0001d752  usbSetLineCoding                           
0001d77c  usbStallEndpoint0                          
0001d7ba  usbStallOEP0                               
00002c6a  wBytesRemainingOnIEP0                      
00002c6c  wBytesRemainingOnOEP0                      
00002c6e  wUsbEventMask                              
00002740  wholeString                                
0001ca12  write                                      


GLOBAL SYMBOLS: SORTED BY Symbol Address 

address   name                                       
-------   ----                                       
00000100  SFRIE1                                     
00000100  SFRIE1_L                                   
00000101  SFRIE1_H                                   
00000102  SFRIFG1                                    
00000102  SFRIFG1_L                                  
00000103  SFRIFG1_H                                  
00000104  SFRRPCR                                    
00000104  SFRRPCR_L                                  
00000105  SFRRPCR_H                                  
00000120  PMMCTL0                                    
00000120  PMMCTL0_L                                  
00000121  PMMCTL0_H                                  
00000122  PMMCTL1                                    
00000122  PMMCTL1_L                                  
00000123  PMMCTL1_H                                  
00000124  SVSMHCTL                                   
00000124  SVSMHCTL_L                                 
00000125  SVSMHCTL_H                                 
00000126  SVSMLCTL                                   
00000126  SVSMLCTL_L                                 
00000127  SVSMLCTL_H                                 
00000128  SVSMIO                                     
00000128  SVSMIO_L                                   
00000129  SVSMIO_H                                   
0000012c  PMMIFG                                     
0000012c  PMMIFG_L                                   
0000012d  PMMIFG_H                                   
0000012e  PMMRIE                                     
0000012e  PMMRIE_L                                   
0000012f  PMMRIE_H                                   
00000130  PM5CTL0                                    
00000130  PM5CTL0_L                                  
00000131  PM5CTL0_H                                  
00000140  FCTL1                                      
00000140  FCTL1_L                                    
00000141  FCTL1_H                                    
00000144  FCTL3                                      
00000144  FCTL3_L                                    
00000145  FCTL3_H                                    
00000146  FCTL4                                      
00000146  FCTL4_L                                    
00000147  FCTL4_H                                    
00000150  CRCDI                                      
00000150  CRCDI_L                                    
00000151  CRCDI_H                                    
00000152  CRCDIRB                                    
00000152  CRCDIRB_L                                  
00000153  CRCDIRB_H                                  
00000154  CRCINIRES                                  
00000154  CRCINIRES_L                                
00000155  CRCINIRES_H                                
00000156  CRCRESR                                    
00000156  CRCRESR_L                                  
00000157  CRCRESR_H                                  
00000158  RCCTL0                                     
00000158  RCCTL0_L                                   
00000159  RCCTL0_H                                   
0000015c  WDTCTL                                     
0000015c  WDTCTL_L                                   
0000015d  WDTCTL_H                                   
00000160  UCSCTL0                                    
00000160  UCSCTL0_L                                  
00000161  UCSCTL0_H                                  
00000162  UCSCTL1                                    
00000162  UCSCTL1_L                                  
00000163  UCSCTL1_H                                  
00000164  UCSCTL2                                    
00000164  UCSCTL2_L                                  
00000165  UCSCTL2_H                                  
00000166  UCSCTL3                                    
00000166  UCSCTL3_L                                  
00000167  UCSCTL3_H                                  
00000168  UCSCTL4                                    
00000168  UCSCTL4_L                                  
00000169  UCSCTL4_H                                  
0000016a  UCSCTL5                                    
0000016a  UCSCTL5_L                                  
0000016b  UCSCTL5_H                                  
0000016c  UCSCTL6                                    
0000016c  UCSCTL6_L                                  
0000016d  UCSCTL6_H                                  
0000016e  UCSCTL7                                    
0000016e  UCSCTL7_L                                  
0000016f  UCSCTL7_H                                  
00000170  UCSCTL8                                    
00000170  UCSCTL8_L                                  
00000171  UCSCTL8_H                                  
00000180  SYSCTL                                     
00000180  SYSCTL_L                                   
00000181  SYSCTL_H                                   
00000182  SYSBSLC                                    
00000182  SYSBSLC_L                                  
00000183  SYSBSLC_H                                  
00000186  SYSJMBC                                    
00000186  SYSJMBC_L                                  
00000187  SYSJMBC_H                                  
00000188  SYSJMBI0                                   
00000188  SYSJMBI0_L                                 
00000189  SYSJMBI0_H                                 
0000018a  SYSJMBI1                                   
0000018a  SYSJMBI1_L                                 
0000018b  SYSJMBI1_H                                 
0000018c  SYSJMBO0                                   
0000018c  SYSJMBO0_L                                 
0000018d  SYSJMBO0_H                                 
0000018e  SYSJMBO1                                   
0000018e  SYSJMBO1_L                                 
0000018f  SYSJMBO1_H                                 
00000190  __STACK_SIZE                               
00000190  __SYSMEM_SIZE                              
00000198  SYSBERRIV                                  
00000198  SYSBERRIV_L                                
00000199  SYSBERRIV_H                                
0000019a  SYSUNIV                                    
0000019a  SYSUNIV_L                                  
0000019b  SYSUNIV_H                                  
0000019c  SYSSNIV                                    
0000019c  SYSSNIV_L                                  
0000019d  SYSSNIV_H                                  
0000019e  SYSRSTIV                                   
0000019e  SYSRSTIV_L                                 
0000019f  SYSRSTIV_H                                 
000001b0  REFCTL0                                    
000001b0  REFCTL0_L                                  
000001b1  REFCTL0_H                                  
000001c0  PMAPKEYID                                  
000001c0  PMAPKEYID_L                                
000001c1  PMAPKEYID_H                                
000001c2  PMAPCTL                                    
000001c2  PMAPCTL_L                                  
000001c3  PMAPCTL_H                                  
000001e0  P4MAP01                                    
000001e0  P4MAP01_L                                  
000001e1  P4MAP01_H                                  
000001e2  P4MAP23                                    
000001e2  P4MAP23_L                                  
000001e3  P4MAP23_H                                  
000001e4  P4MAP45                                    
000001e4  P4MAP45_L                                  
000001e5  P4MAP45_H                                  
000001e6  P4MAP67                                    
000001e6  P4MAP67_L                                  
000001e7  P4MAP67_H                                  
00000200  PAIN                                       
00000200  PAIN_L                                     
00000201  PAIN_H                                     
00000202  PAOUT                                      
00000202  PAOUT_L                                    
00000203  PAOUT_H                                    
00000204  PADIR                                      
00000204  PADIR_L                                    
00000205  PADIR_H                                    
00000206  PAREN                                      
00000206  PAREN_L                                    
00000207  PAREN_H                                    
00000208  PADS                                       
00000208  PADS_L                                     
00000209  PADS_H                                     
0000020a  PASEL                                      
0000020a  PASEL_L                                    
0000020b  PASEL_H                                    
0000020e  P1IV                                       
00000218  PAIES                                      
00000218  PAIES_L                                    
00000219  PAIES_H                                    
0000021a  PAIE                                       
0000021a  PAIE_L                                     
0000021b  PAIE_H                                     
0000021c  PAIFG                                      
0000021c  PAIFG_L                                    
0000021d  PAIFG_H                                    
0000021e  P2IV                                       
00000220  PBIN                                       
00000220  PBIN_L                                     
00000221  PBIN_H                                     
00000222  PBOUT                                      
00000222  PBOUT_L                                    
00000223  PBOUT_H                                    
00000224  PBDIR                                      
00000224  PBDIR_L                                    
00000225  PBDIR_H                                    
00000226  PBREN                                      
00000226  PBREN_L                                    
00000227  PBREN_H                                    
00000228  PBDS                                       
00000228  PBDS_L                                     
00000229  PBDS_H                                     
0000022a  PBSEL                                      
0000022a  PBSEL_L                                    
0000022b  PBSEL_H                                    
00000240  PCIN                                       
00000240  PCIN_L                                     
00000241  PCIN_H                                     
00000242  PCOUT                                      
00000242  PCOUT_L                                    
00000243  PCOUT_H                                    
00000244  PCDIR                                      
00000244  PCDIR_L                                    
00000245  PCDIR_H                                    
00000246  PCREN                                      
00000246  PCREN_L                                    
00000247  PCREN_H                                    
00000248  PCDS                                       
00000248  PCDS_L                                     
00000249  PCDS_H                                     
0000024a  PCSEL                                      
0000024a  PCSEL_L                                    
0000024b  PCSEL_H                                    
00000260  PDIN                                       
00000260  PDIN_L                                     
00000261  PDIN_H                                     
00000262  PDOUT                                      
00000262  PDOUT_L                                    
00000263  PDOUT_H                                    
00000264  PDDIR                                      
00000264  PDDIR_L                                    
00000265  PDDIR_H                                    
00000266  PDREN                                      
00000266  PDREN_L                                    
00000267  PDREN_H                                    
00000268  PDDS                                       
00000268  PDDS_L                                     
00000269  PDDS_H                                     
0000026a  PDSEL                                      
0000026a  PDSEL_L                                    
0000026b  PDSEL_H                                    
00000320  PJIN                                       
00000320  PJIN_L                                     
00000321  PJIN_H                                     
00000322  PJOUT                                      
00000322  PJOUT_L                                    
00000323  PJOUT_H                                    
00000324  PJDIR                                      
00000324  PJDIR_L                                    
00000325  PJDIR_H                                    
00000326  PJREN                                      
00000326  PJREN_L                                    
00000327  PJREN_H                                    
00000328  PJDS                                       
00000328  PJDS_L                                     
00000329  PJDS_H                                     
00000340  TA0CTL                                     
00000342  TA0CCTL0                                   
00000344  TA0CCTL1                                   
00000346  TA0CCTL2                                   
00000348  TA0CCTL3                                   
0000034a  TA0CCTL4                                   
00000350  TA0R                                       
00000352  TA0CCR0                                    
00000354  TA0CCR1                                    
00000356  TA0CCR2                                    
00000358  TA0CCR3                                    
0000035a  TA0CCR4                                    
00000360  TA0EX0                                     
0000036e  TA0IV                                      
00000380  TA1CTL                                     
00000382  TA1CCTL0                                   
00000384  TA1CCTL1                                   
00000386  TA1CCTL2                                   
00000390  TA1R                                       
00000392  TA1CCR0                                    
00000394  TA1CCR1                                    
00000396  TA1CCR2                                    
000003a0  TA1EX0                                     
000003ae  TA1IV                                      
000003c0  TB0CTL                                     
000003c2  TB0CCTL0                                   
000003c4  TB0CCTL1                                   
000003c6  TB0CCTL2                                   
000003c8  TB0CCTL3                                   
000003ca  TB0CCTL4                                   
000003cc  TB0CCTL5                                   
000003ce  TB0CCTL6                                   
000003d0  TB0R                                       
000003d2  TB0CCR0                                    
000003d4  TB0CCR1                                    
000003d6  TB0CCR2                                    
000003d8  TB0CCR3                                    
000003da  TB0CCR4                                    
000003dc  TB0CCR5                                    
000003de  TB0CCR6                                    
000003e0  TB0EX0                                     
000003ee  TB0IV                                      
00000400  TA2CTL                                     
00000402  TA2CCTL0                                   
00000404  TA2CCTL1                                   
00000406  TA2CCTL2                                   
00000410  TA2R                                       
00000412  TA2CCR0                                    
00000414  TA2CCR1                                    
00000416  TA2CCR2                                    
00000420  TA2EX0                                     
0000042e  TA2IV                                      
000004a0  RTCCTL01                                   
000004a0  RTCCTL01_L                                 
000004a1  RTCCTL01_H                                 
000004a2  RTCCTL23                                   
000004a2  RTCCTL23_L                                 
000004a3  RTCCTL23_H                                 
000004a8  RTCPS0CTL                                  
000004a8  RTCPS0CTL_L                                
000004a9  RTCPS0CTL_H                                
000004aa  RTCPS1CTL                                  
000004aa  RTCPS1CTL_L                                
000004ab  RTCPS1CTL_H                                
000004ac  RTCPS                                      
000004ac  RTCPS_L                                    
000004ad  RTCPS_H                                    
000004ae  RTCIV                                      
000004b0  RTCTIM0                                    
000004b0  RTCTIM0_L                                  
000004b1  RTCTIM0_H                                  
000004b2  RTCTIM1                                    
000004b2  RTCTIM1_L                                  
000004b3  RTCTIM1_H                                  
000004b4  RTCDATE                                    
000004b4  RTCDATE_L                                  
000004b5  RTCDATE_H                                  
000004b6  RTCYEAR                                    
000004b6  RTCYEAR_L                                  
000004b7  RTCYEAR_H                                  
000004b8  RTCAMINHR                                  
000004b8  RTCAMINHR_L                                
000004b9  RTCAMINHR_H                                
000004ba  RTCADOWDAY                                 
000004ba  RTCADOWDAY_L                               
000004bb  RTCADOWDAY_H                               
000004c0  MPY                                        
000004c0  MPY_L                                      
000004c1  MPY_H                                      
000004c2  MPYS                                       
000004c2  MPYS_L                                     
000004c3  MPYS_H                                     
000004c4  MAC                                        
000004c4  MAC_L                                      
000004c5  MAC_H                                      
000004c6  MACS                                       
000004c6  MACS_L                                     
000004c7  MACS_H                                     
000004c8  OP2                                        
000004c8  OP2_L                                      
000004c9  OP2_H                                      
000004ca  RESLO                                      
000004ca  RESLO_L                                    
000004cb  RESLO_H                                    
000004cc  RESHI                                      
000004cc  RESHI_L                                    
000004cd  RESHI_H                                    
000004ce  SUMEXT                                     
000004ce  SUMEXT_L                                   
000004cf  SUMEXT_H                                   
000004d0  MPY32L                                     
000004d0  MPY32L_L                                   
000004d1  MPY32L_H                                   
000004d2  MPY32H                                     
000004d2  MPY32H_L                                   
000004d3  MPY32H_H                                   
000004d4  MPYS32L                                    
000004d4  MPYS32L_L                                  
000004d5  MPYS32L_H                                  
000004d6  MPYS32H                                    
000004d6  MPYS32H_L                                  
000004d7  MPYS32H_H                                  
000004d8  MAC32L                                     
000004d8  MAC32L_L                                   
000004d9  MAC32L_H                                   
000004da  MAC32H                                     
000004da  MAC32H_L                                   
000004db  MAC32H_H                                   
000004dc  MACS32L                                    
000004dc  MACS32L_L                                  
000004dd  MACS32L_H                                  
000004de  MACS32H                                    
000004de  MACS32H_L                                  
000004df  MACS32H_H                                  
000004e0  OP2L                                       
000004e0  OP2L_L                                     
000004e1  OP2L_H                                     
000004e2  OP2H                                       
000004e2  OP2H_L                                     
000004e3  OP2H_H                                     
000004e4  RES0                                       
000004e4  RES0_L                                     
000004e5  RES0_H                                     
000004e6  RES1                                       
000004e6  RES1_L                                     
000004e7  RES1_H                                     
000004e8  RES2                                       
000004e8  RES2_L                                     
000004e9  RES2_H                                     
000004ea  RES3                                       
000004ea  RES3_L                                     
000004eb  RES3_H                                     
000004ec  MPY32CTL0                                  
000004ec  MPY32CTL0_L                                
000004ed  MPY32CTL0_H                                
00000500  DMACTL0                                    
00000500  DMACTL0_L                                  
00000501  DMACTL0_H                                  
00000502  DMACTL1                                    
00000502  DMACTL1_L                                  
00000503  DMACTL1_H                                  
00000504  DMACTL2                                    
00000504  DMACTL2_L                                  
00000505  DMACTL2_H                                  
00000506  DMACTL3                                    
00000506  DMACTL3_L                                  
00000507  DMACTL3_H                                  
00000508  DMACTL4                                    
00000508  DMACTL4_L                                  
00000509  DMACTL4_H                                  
0000050e  DMAIV                                      
0000050e  DMAIV_L                                    
0000050f  DMAIV_H                                    
00000510  DMA0CTL                                    
00000510  DMA0CTL_L                                  
00000511  DMA0CTL_H                                  
00000512  DMA0SA                                     
00000512  DMA0SAL                                    
00000514  DMA0SAH                                    
00000516  DMA0DA                                     
00000516  DMA0DAL                                    
00000518  DMA0DAH                                    
0000051a  DMA0SZ                                     
00000520  DMA1CTL                                    
00000520  DMA1CTL_L                                  
00000521  DMA1CTL_H                                  
00000522  DMA1SA                                     
00000522  DMA1SAL                                    
00000524  DMA1SAH                                    
00000526  DMA1DA                                     
00000526  DMA1DAL                                    
00000528  DMA1DAH                                    
0000052a  DMA1SZ                                     
00000530  DMA2CTL                                    
00000530  DMA2CTL_L                                  
00000531  DMA2CTL_H                                  
00000532  DMA2SA                                     
00000532  DMA2SAL                                    
00000534  DMA2SAH                                    
00000536  DMA2DA                                     
00000536  DMA2DAL                                    
00000538  DMA2DAH                                    
0000053a  DMA2SZ                                     
000005c0  UCA0CTLW0                                  
000005c0  UCA0CTLW0_L                                
000005c1  UCA0CTLW0_H                                
000005c6  UCA0BRW                                    
000005c6  UCA0BRW_L                                  
000005c7  UCA0BRW_H                                  
000005c8  UCA0MCTL                                   
000005ca  UCA0STAT                                   
000005cc  UCA0RXBUF                                  
000005ce  UCA0TXBUF                                  
000005d0  UCA0ABCTL                                  
000005d2  UCA0IRCTL                                  
000005d2  UCA0IRCTL_L                                
000005d3  UCA0IRCTL_H                                
000005dc  UCA0ICTL                                   
000005dc  UCA0ICTL_L                                 
000005dd  UCA0ICTL_H                                 
000005de  UCA0IV                                     
000005e0  UCB0CTLW0                                  
000005e0  UCB0CTLW0_L                                
000005e1  UCB0CTLW0_H                                
000005e6  UCB0BRW                                    
000005e6  UCB0BRW_L                                  
000005e7  UCB0BRW_H                                  
000005ea  UCB0STAT                                   
000005ec  UCB0RXBUF                                  
000005ee  UCB0TXBUF                                  
000005f0  UCB0I2COA                                  
000005f0  UCB0I2COA_L                                
000005f1  UCB0I2COA_H                                
000005f2  UCB0I2CSA                                  
000005f2  UCB0I2CSA_L                                
000005f3  UCB0I2CSA_H                                
000005fc  UCB0ICTL                                   
000005fc  UCB0ICTL_L                                 
000005fd  UCB0ICTL_H                                 
000005fe  UCB0IV                                     
00000600  UCA1CTLW0                                  
00000600  UCA1CTLW0_L                                
00000601  UCA1CTLW0_H                                
00000606  UCA1BRW                                    
00000606  UCA1BRW_L                                  
00000607  UCA1BRW_H                                  
00000608  UCA1MCTL                                   
0000060a  UCA1STAT                                   
0000060c  UCA1RXBUF                                  
0000060e  UCA1TXBUF                                  
00000610  UCA1ABCTL                                  
00000612  UCA1IRCTL                                  
00000612  UCA1IRCTL_L                                
00000613  UCA1IRCTL_H                                
0000061c  UCA1ICTL                                   
0000061c  UCA1ICTL_L                                 
0000061d  UCA1ICTL_H                                 
0000061e  UCA1IV                                     
00000620  UCB1CTLW0                                  
00000620  UCB1CTLW0_L                                
00000621  UCB1CTLW0_H                                
00000626  UCB1BRW                                    
00000626  UCB1BRW_L                                  
00000627  UCB1BRW_H                                  
0000062a  UCB1STAT                                   
0000062c  UCB1RXBUF                                  
0000062e  UCB1TXBUF                                  
00000630  UCB1I2COA                                  
00000630  UCB1I2COA_L                                
00000631  UCB1I2COA_H                                
00000632  UCB1I2CSA                                  
00000632  UCB1I2CSA_L                                
00000633  UCB1I2CSA_H                                
0000063c  UCB1ICTL                                   
0000063c  UCB1ICTL_L                                 
0000063d  UCB1ICTL_H                                 
0000063e  UCB1IV                                     
00000700  ADC12CTL0                                  
00000700  ADC12CTL0_L                                
00000701  ADC12CTL0_H                                
00000702  ADC12CTL1                                  
00000702  ADC12CTL1_L                                
00000703  ADC12CTL1_H                                
00000704  ADC12CTL2                                  
00000704  ADC12CTL2_L                                
00000705  ADC12CTL2_H                                
0000070a  ADC12IFG                                   
0000070a  ADC12IFG_L                                 
0000070b  ADC12IFG_H                                 
0000070c  ADC12IE                                    
0000070c  ADC12IE_L                                  
0000070d  ADC12IE_H                                  
0000070e  ADC12IV                                    
0000070e  ADC12IV_L                                  
0000070f  ADC12IV_H                                  
00000710  ADC12MCTL0                                 
00000711  ADC12MCTL1                                 
00000712  ADC12MCTL2                                 
00000713  ADC12MCTL3                                 
00000714  ADC12MCTL4                                 
00000715  ADC12MCTL5                                 
00000716  ADC12MCTL6                                 
00000717  ADC12MCTL7                                 
00000718  ADC12MCTL8                                 
00000719  ADC12MCTL9                                 
0000071a  ADC12MCTL10                                
0000071b  ADC12MCTL11                                
0000071c  ADC12MCTL12                                
0000071d  ADC12MCTL13                                
0000071e  ADC12MCTL14                                
0000071f  ADC12MCTL15                                
00000720  ADC12MEM0                                  
00000720  ADC12MEM0_L                                
00000721  ADC12MEM0_H                                
00000722  ADC12MEM1                                  
00000722  ADC12MEM1_L                                
00000723  ADC12MEM1_H                                
00000724  ADC12MEM2                                  
00000724  ADC12MEM2_L                                
00000725  ADC12MEM2_H                                
00000726  ADC12MEM3                                  
00000726  ADC12MEM3_L                                
00000727  ADC12MEM3_H                                
00000728  ADC12MEM4                                  
00000728  ADC12MEM4_L                                
00000729  ADC12MEM4_H                                
0000072a  ADC12MEM5                                  
0000072a  ADC12MEM5_L                                
0000072b  ADC12MEM5_H                                
0000072c  ADC12MEM6                                  
0000072c  ADC12MEM6_L                                
0000072d  ADC12MEM6_H                                
0000072e  ADC12MEM7                                  
0000072e  ADC12MEM7_L                                
0000072f  ADC12MEM7_H                                
00000730  ADC12MEM8                                  
00000730  ADC12MEM8_L                                
00000731  ADC12MEM8_H                                
00000732  ADC12MEM9                                  
00000732  ADC12MEM9_L                                
00000733  ADC12MEM9_H                                
00000734  ADC12MEM10                                 
00000734  ADC12MEM10_L                               
00000735  ADC12MEM10_H                               
00000736  ADC12MEM11                                 
00000736  ADC12MEM11_L                               
00000737  ADC12MEM11_H                               
00000738  ADC12MEM12                                 
00000738  ADC12MEM12_L                               
00000739  ADC12MEM12_H                               
0000073a  ADC12MEM13                                 
0000073a  ADC12MEM13_L                               
0000073b  ADC12MEM13_H                               
0000073c  ADC12MEM14                                 
0000073c  ADC12MEM14_L                               
0000073d  ADC12MEM14_H                               
0000073e  ADC12MEM15                                 
0000073e  ADC12MEM15_L                               
0000073f  ADC12MEM15_H                               
000008c0  CBCTL0                                     
000008c0  CBCTL0_L                                   
000008c1  CBCTL0_H                                   
000008c2  CBCTL1                                     
000008c2  CBCTL1_L                                   
000008c3  CBCTL1_H                                   
000008c4  CBCTL2                                     
000008c4  CBCTL2_L                                   
000008c5  CBCTL2_H                                   
000008c6  CBCTL3                                     
000008c6  CBCTL3_L                                   
000008c7  CBCTL3_H                                   
000008cc  CBINT                                      
000008cc  CBINT_L                                    
000008cd  CBINT_H                                    
000008ce  CBIV                                       
00000900  USBKEYID                                   
00000900  USBKEYID_L                                 
00000901  USBKEYID_H                                 
00000902  USBCNF                                     
00000902  USBCNF_L                                   
00000903  USBCNF_H                                   
00000904  USBPHYCTL                                  
00000904  USBPHYCTL_L                                
00000905  USBPHYCTL_H                                
00000908  USBPWRCTL                                  
00000908  USBPWRCTL_L                                
00000909  USBPWRCTL_H                                
00000910  USBPLLCTL                                  
00000910  USBPLLCTL_L                                
00000911  USBPLLCTL_H                                
00000912  USBPLLDIVB                                 
00000912  USBPLLDIVB_L                               
00000913  USBPLLDIVB_H                               
00000914  USBPLLIR                                   
00000914  USBPLLIR_L                                 
00000915  USBPLLIR_H                                 
00000920  USBIEPCNF_0                                
00000920  tEndPoint0DescriptorBlock                  
00000921  USBIEPCNT_0                                
00000922  USBOEPCNF_0                                
00000923  USBOEPCNT_0                                
0000092e  USBIEPIE                                   
0000092f  USBOEPIE                                   
00000930  USBIEPIFG                                  
00000931  USBOEPIFG                                  
00000932  USBVECINT                                  
00000932  USBVECINT_L                                
00000933  USBVECINT_H                                
00000936  USBMAINT                                   
00000936  USBMAINT_L                                 
00000937  USBMAINT_H                                 
00000938  USBTSREG                                   
00000938  USBTSREG_L                                 
00000939  USBTSREG_H                                 
0000093a  USBFN                                      
0000093a  USBFN_L                                    
0000093b  USBFN_H                                    
0000093c  USBCTL                                     
0000093d  USBIE                                      
0000093e  USBIFG                                     
0000093f  USBFUNADR                                  
00001c00  USBSTABUFF                                 
00001c00  pbXBufferAddressEp1                        
00001c40  pbYBufferAddressEp1                        
00001c80  pbXBufferAddressEp81                       
00001cc0  pbYBufferAddressEp81                       
00001d00  pbXBufferAddressEp2                        
00001d40  pbYBufferAddressEp2                        
00001d80  pbXBufferAddressEp82                       
00001dc0  pbYBufferAddressEp82                       
00001e00  pbXBufferAddressEp3                        
00001e40  pbYBufferAddressEp3                        
00001e80  pbXBufferAddressEp83                       
00001ec0  pbYBufferAddressEp83                       
00001f00  pbXBufferAddressEp4                        
00001f40  pbYBufferAddressEp4                        
00001f80  pbXBufferAddressEp84                       
00001fc0  pbYBufferAddressEp84                       
00002000  pbXBufferAddressEp5                        
00002040  pbYBufferAddressEp5                        
00002080  pbXBufferAddressEp85                       
000020c0  pbYBufferAddressEp85                       
00002100  pbXBufferAddressEp6                        
00002140  pbYBufferAddressEp6                        
00002180  pbXBufferAddressEp86                       
000021c0  pbYBufferAddressEp86                       
00002200  pbXBufferAddressEp7                        
00002240  pbYBufferAddressEp7                        
00002280  pbXBufferAddressEp87                       
000022c0  pbYBufferAddressEp87                       
0000236f  USBTOPBUFF                                 
00002370  USBOEP0BUF                                 
00002370  abOEP0Buffer                               
00002378  USBIEP0BUF                                 
00002378  abIEP0Buffer                               
00002380  USBSUBLK                                   
00002380  tSetupPacket                               
00002388  USBOEPCNF_1                                
00002388  tOutputEndPointDescriptorBlock             
00002389  USBOEPBBAX_1                               
0000238a  USBOEPBCTX_1                               
0000238d  USBOEPBBAY_1                               
0000238e  USBOEPBCTY_1                               
0000238f  USBOEPSIZXY_1                              
00002390  USBOEPCNF_2                                
00002391  USBOEPBBAX_2                               
00002392  USBOEPBCTX_2                               
00002395  USBOEPBBAY_2                               
00002396  USBOEPBCTY_2                               
00002397  USBOEPSIZXY_2                              
00002398  USBOEPCNF_3                                
00002399  USBOEPBBAX_3                               
0000239a  USBOEPBCTX_3                               
0000239d  USBOEPBBAY_3                               
0000239e  USBOEPBCTY_3                               
0000239f  USBOEPSIZXY_3                              
000023a0  USBOEPCNF_4                                
000023a1  USBOEPBBAX_4                               
000023a2  USBOEPBCTX_4                               
000023a5  USBOEPBBAY_4                               
000023a6  USBOEPBCTY_4                               
000023a7  USBOEPSIZXY_4                              
000023a8  USBOEPCNF_5                                
000023a9  USBOEPBBAX_5                               
000023aa  USBOEPBCTX_5                               
000023ad  USBOEPBBAY_5                               
000023ae  USBOEPBCTY_5                               
000023af  USBOEPSIZXY_5                              
000023b0  USBOEPCNF_6                                
000023b1  USBOEPBBAX_6                               
000023b2  USBOEPBCTX_6                               
000023b5  USBOEPBBAY_6                               
000023b6  USBOEPBCTY_6                               
000023b7  USBOEPSIZXY_6                              
000023b8  USBOEPCNF_7                                
000023b9  USBOEPBBAX_7                               
000023ba  USBOEPBCTX_7                               
000023bd  USBOEPBBAY_7                               
000023be  USBOEPBCTY_7                               
000023bf  USBOEPSIZXY_7                              
000023c8  USBIEPCNF_1                                
000023c8  tInputEndPointDescriptorBlock              
000023c9  USBIEPBBAX_1                               
000023ca  USBIEPBCTX_1                               
000023cd  USBIEPBBAY_1                               
000023ce  USBIEPBCTY_1                               
000023cf  USBIEPSIZXY_1                              
000023d0  USBIEPCNF_2                                
000023d1  USBIEPBBAX_2                               
000023d2  USBIEPBCTX_2                               
000023d5  USBIEPBBAY_2                               
000023d6  USBIEPBCTY_2                               
000023d7  USBIEPSIZXY_2                              
000023d8  USBIEPCNF_3                                
000023d9  USBIEPBBAX_3                               
000023da  USBIEPBCTX_3                               
000023dd  USBIEPBBAY_3                               
000023de  USBIEPBCTY_3                               
000023df  USBIEPSIZXY_3                              
000023e0  USBIEPCNF_4                                
000023e1  USBIEPBBAX_4                               
000023e2  USBIEPBCTX_4                               
000023e5  USBIEPBBAY_4                               
000023e6  USBIEPBCTY_4                               
000023e7  USBIEPSIZXY_4                              
000023e8  USBIEPCNF_5                                
000023e9  USBIEPBBAX_5                               
000023ea  USBIEPBCTX_5                               
000023ed  USBIEPBBAY_5                               
000023ee  USBIEPBCTY_5                               
000023ef  USBIEPSIZXY_5                              
000023f0  USBIEPCNF_6                                
000023f1  USBIEPBBAX_6                               
000023f2  USBIEPBCTX_6                               
000023f5  USBIEPBBAY_6                               
000023f6  USBIEPBCTY_6                               
000023f7  USBIEPSIZXY_6                              
000023f8  USBIEPCNF_7                                
000023f9  USBIEPBBAX_7                               
000023fa  USBIEPBCTX_7                               
000023fd  USBIEPBBAY_7                               
000023fe  USBIEPBCTY_7                               
000023ff  USBIEPSIZXY_7                              
00002400  _ftable                                    
00002578  _Denorm                                    
00002588  _Eps                                       
00002598  _Hugeval                                   
000025a8  _Inf                                       
000025b8  _Nan                                       
000025c8  _Snan                                      
000025d8  _Rteps                                     
000025e8  _Xbig                                      
000025f0  _Zero                                      
00002670  ADS126xRegisterNames                       
000026dc  outString                                  
00002740  wholeString                                
000027a4  scr_mux_norm_strings                       
000027e4  scr_speed_norm_strings                     
00002860  scr_idacdir_norm_strings                   
00002890  scr_idacmag_norm_strings                   
000028bc  scr_gpio_norm_strings                      
000028dc  scr_pga_norm_strings                       
000028fc  tempString                                 
00002916  scr_adc2ref_norm_strings                   
0000292a  scr_filter_norm_strings                    
0000293e  scr_refn_norm_strings                      
00002952  scr_refp_norm_strings                      
00002978  scr_adc2speed_norm_strings                 
00002988  UCS_XT1ClockFrequency                      
0000298c  UCS_XT2ClockFrequency                      
00002990  _Fenv                                      
00002994  _Tls_setup__Fenv                           
00002999  bFunctionSuspended                         
0000299a  bEnumerationStatus                         
0000299c  VERSION                                    
000029a0  __TI_cleanup_ptr                           
000029a4  __TI_dtors_ptr                             
000029a8  _lock                                      
000029ac  _unlock                                    
000029b0  __TI_ft_end                                
000029b2  _Errno                                     
000029b6  g_DRDY_flag                                
000029b7  g_bCDCDataReceived_event                   
000029b8  _sys_memory                                
00002b48  __TI_tmpnams                               
00002be8  abramSerialStringDescriptor                
00002c38  abUsbRequestIncomingData                   
00002c40  abUsbRequestReturnData                     
00002c50  USB_RX_memcpy                              
00002c54  USB_TX_memcpy                              
00002c6a  wBytesRemainingOnIEP0                      
00002c6c  wBytesRemainingOnOEP0                      
00002c6e  wUsbEventMask                              
00002c73  bStatusAction                              
00002c74  _CIOBUF_                                   
00004270  _stack                                     
00004400  __STACK_END                                
00004400  iUsbInterruptHandler                       
000045b0  UNMI_ISR                                   
000045fc  PORT1_ISR                                  
0000461a  _c_int00_noargs                            
00004636  TIMER0_A0_ISR                              
00004644  __TI_ISR_TRAP                              
0000978a  tUsbRequestList                            
00009894  _ctypes_                                   
00009995  MinNumADCReadings                          
00009a36  abromStringDescriptor                      
00009acc  abromConfigurationDescriptorGroup          
00009b6e  abromDeviceDescriptor                      
00009b90  stUsbHandle                                
00009e2a  __TI_Handler_Table_Base                    
00009e36  __TI_Handler_Table_Limit                   
00009e42  __TI_CINIT_Base                            
00009e5a  __TI_CINIT_Limit                           
0000ffd2  __TI_int41                                 
0000ffd4  __TI_int42                                 
0000ffd6  __TI_int43                                 
0000ffd8  __TI_int44                                 
0000ffda  __TI_int45                                 
0000ffdc  __TI_int46                                 
0000ffde  __TI_int47                                 
0000ffe0  __TI_int48                                 
0000ffe2  __TI_int49                                 
0000ffe4  __TI_int50                                 
0000ffe6  __TI_int51                                 
0000ffe8  __TI_int52                                 
0000ffea  __TI_int53                                 
0000ffec  __TI_int54                                 
0000ffee  __TI_int55                                 
0000fff0  __TI_int56                                 
0000fff2  __TI_int57                                 
0000fff4  __TI_int58                                 
0000fff6  __TI_int59                                 
0000fff8  __TI_int60                                 
0000fffa  __TI_int61                                 
0000fffc  __TI_int62                                 
0000fffe  _reset_vector                              
00010000  show_parms                                 
00010caa  USBCDC_receiveData                         
0001164c  __TI_frcdivd                               
000126c8  __mspabi_divull                            
00012a62  _Exp                                       
00012dea  CdcToHostFromBuffer                        
0001344e  __TI_frcmpyd                               
00013732  __mspabi_addd                              
00013a0a  set_gpio                                   
00013cd0  console                                    
00013f84  set_vref                                   
00014224  __mspabi_mpyd                              
000144a6  CdcToBufferFromHost                        
00014980  __TI_frcaddd                               
00014bd2  __mspabi_divd                              
00015436  __TI_printfi                               
0001583a  GPIO_setAsInputPin                         
00015a20  USB_reset                                  
00015bf8  set_idac                                   
00015dca  strtoul                                    
00015f96  retInString                                
00016326  GPIO_setAsOutputPin                        
000164dc  GPIO_setAsPeripheralModuleFunctionInputPin 
00016692  GPIO_setAsPeripheralModuleFunctionOutputPin
00016b9a  _Dscale                                    
00016d38  set_mux                                    
0001705a  GPIO_setOutputHighOnPin                    
000171e0  GPIO_setOutputLowOnPin                     
00017366  GPIO_toggleOutputOnPin                     
000174ec  UCS_clockSignalInit                        
0001765c  hex2asc                                    
00017bd4  USB_InitSerialStringDescriptor             
00017d18  CopyUsbToBuff                              
00017e4e  UCS_initFLL                                
00017f7c  DMA_init                                   
000180a2  adc2_mux                                   
000181c8  initPorts                                  
000182ee  USBCDC_intfStatus                          
0001851e  PMM_setVCoreUp                             
0001872e  ADS126xReadData                            
00018834  _Dnorm                                     
00018934  GPIO_interruptEdgeSelect                   
00018c26  usbDecodeAndProcessUsbRequest              
00018d20  USB_enable                                 
00018e18  USCI_B_SPI_masterInit                      
00018f0e  USBCDC_bytesInUSBBuffer                    
00018ffe  exp2                                       
000190ee  fputs                                      
000191de  set_datarate                               
000192cc  set_register                               
000193b8  setvbuf                                    
00019498  set_chop                                   
00019574  set_conv_mode                              
00019650  __mspabi_cmpd                              
00019728  set_filter                                 
000197fe  set_bias                                   
0001999c  GPIO_clearInterruptFlag                    
00019a68  GPIO_disableInterrupt                      
00019b34  GPIO_enableInterrupt                       
00019cc6  USBtask                                    
00019d8a  USBCDC_sendData                            
00019f0c  PMM_setVCoreDown                           
00019fcc  set_exc                                    
0001a08a  USB_determineFreq                          
0001a144  malloc                                     
0001a1fe  __TI_renormd                               
0001a2b0  UCS_LFXT1Start                             
0001a35e  cdcSendDataWaitTilDone                     
0001a40c  USB_init                                   
0001a4b6  adc2_startstop                             
0001a608  cdcReceiveDataInBuffer                     
0001a6ae  usbGetEndpointStatus                       
0001a754  set_pga                                    
0001a7f8  cdcSendDataInBackground                    
0001a89a  usbGetLineCoding                           
0001a93a  HOSTlseek                                  
0001aa76  PMM_setVCore                               
0001ab10  run_demo                                   
0001aba8  USB_connectionState                        
0001ac3e  adc2_datarate                              
0001acd4  adc2_reference                             
0001ad6a  __mspabi_fltlid                            
0001ae92  TLV_getInfo                                
0001afb2  free                                       
0001b040  adc2_pga                                   
0001b154  ldexp                                      
0001b1da  DMA_setDstAddress                          
0001b25c  PWRVBUSoffHandler                          
0001b2de  ltoa                                       
0001b35e  usbSendNextPacketOnIEP0                    
0001b3de  DMA_setSrcAddress                          
0001b45c  __TI_wrt_ok                                
0001b4da  memcpyDMA                                  
0001b5ce  Handler_SetLineCoding                      
0001b6be  usbGetStringDescriptor                     
0001b736  __mspabi_fltuld                            
0001b7ac  HOSTrename                                 
0001b820  _Dunscale                                  
0001b892  PWRVBUSonHandler                           
0001b902  __TI_closefile                             
0001b972  HOSTopen                                   
0001b9e0  _auto_init_hold_wdt                        
0001ba4c  adc2                                       
0001bab8  HOSTwrite                                  
0001bb22  UCS_XT2StartWithTimeout                    
0001bb8c  fseek                                      
0001bbf6  usbReceiveNextPacketOnOEP0                 
0001bc60  HOSTread                                   
0001bd30  ADS126xReadRegister                        
0001bd96  __mspabi_fixdli                            
0001be62  __TI_doflush                               
0001bec6  initClocks                                 
0001bf2a  ADS126xWriteRegister                       
0001bf8c  atoi                                       
0001bfee  snprintf                                   
0001c050  SetupPacketInterruptHandler                
0001c0ac  close                                      
0001c160  run_adc2_demo                              
0001c1ba  fflush                                     
0001c212  memcpyV                                    
0001c26a  __mspabi_divul                             
0001c26a  __mspabi_remul                             
0001c2c2  usbSetEndpointFeature                      
0001c318  initSPI                                    
0001c36c  usbClearEndpointFeature                    
0001c3c0  _Dclass                                    
0001c410  UCS_initFLLSettle                          
0001c4ac  HOSTclose                                  
0001c4f8  CdcResetData                               
0001c542  USB_setup                                  
0001c58c  print2Console                              
0001c5d4  HOSTunlink                                 
0001c660  sprintf                                    
0001c6a4  frexp                                      
0001c6e6  minit                                      
0001c728  PressANYkeytoContinue                      
0001c768  USB_connectionInfo                         
0001c7a8  USB_initMemcpy                             
0001c7e8  __mspabi_divli                             
0001c7e8  __mspabi_remli                             
0001c866  __mspabi_sral_15                           
0001c86a  __mspabi_sral_14                           
0001c86e  __mspabi_sral_13                           
0001c872  __mspabi_sral_12                           
0001c876  __mspabi_sral_11                           
0001c87a  __mspabi_sral_10                           
0001c87e  __mspabi_sral_9                            
0001c882  __mspabi_sral_8                            
0001c886  __mspabi_sral_7                            
0001c88a  __mspabi_sral_6                            
0001c88e  __mspabi_sral_5                            
0001c892  __mspabi_sral_4                            
0001c896  __mspabi_sral_3                            
0001c89a  __mspabi_sral_2                            
0001c89e  __mspabi_sral_1                            
0001c8a4  __mspabi_slll_15                           
0001c8a8  __mspabi_slll_14                           
0001c8ac  __mspabi_slll_13                           
0001c8b0  __mspabi_slll_12                           
0001c8b4  __mspabi_slll_11                           
0001c8b8  __mspabi_slll_10                           
0001c8bc  __mspabi_slll_9                            
0001c8c0  __mspabi_slll_8                            
0001c8c4  __mspabi_slll_7                            
0001c8c8  __mspabi_slll_6                            
0001c8cc  __mspabi_slll_5                            
0001c8d0  __mspabi_slll_4                            
0001c8d4  __mspabi_slll_3                            
0001c8d8  __mspabi_slll_2                            
0001c8dc  __mspabi_slll_1                            
0001c8e2  __mspabi_srll_15                           
0001c8e6  __mspabi_srll_14                           
0001c8ea  __mspabi_srll_13                           
0001c8ee  __mspabi_srll_12                           
0001c8f2  __mspabi_srll_11                           
0001c8f6  __mspabi_srll_10                           
0001c8fa  __mspabi_srll_9                            
0001c8fe  __mspabi_srll_8                            
0001c902  __mspabi_srll_7                            
0001c906  __mspabi_srll_6                            
0001c90a  __mspabi_srll_5                            
0001c90e  __mspabi_srll_4                            
0001c912  __mspabi_srll_3                            
0001c916  __mspabi_srll_2                            
0001c91a  __mspabi_srll_1                            
0001c920  lseek                                      
0001c95e  ADS126xXferByte                            
0001c99a  OEP0InterruptHandler                       
0001c9d6  UCS_XT2Start                               
0001ca12  write                                      
0001ca4e  USCI_B_SPI_disableInterrupt                
0001ca88  __mspabi_sllll                             
0001cac2  __mspabi_srlll                             
0001cafc  show_version                               
0001cb36  set_adc_CS                                 
0001cb6e  set_adc_START                              
0001cba6  signal                                     
0001cbde  usbSendDataPacketOnEP0                     
0001cc16  _Feraise                                   
0001cc4c  __TI_cleanup                               
0001cc82  __TI_writemsg                              
0001ccb4  C$$IO$$                                    
0001ccee  WDT_A_hold                                 
0001cd22  feraiseexcept                              
0001cd56  usbDisableInEndpointInterrupt              
0001cd8a  usbDisableOutEndpointInterrupt             
0001cdbe  UCS_getSMCLK                               
0001cdf0  __TI_readmsg                               
0001ce22  __mspabi_subd                              
0001ce54  main                                       
0001ce86  raise                                      
0001ceb8  strncpy                                    
0001ceea  usbGetDeviceStatus                         
0001cf1c  usbSetConfiguration                        
0001cf4e  DMA_disableTransfers                       
0001cf7e  DMA_enableTransfers                        
0001cfae  UCS_setExternalClockSource                 
0001cfde  USB_suspend                                
0001d00e  remove                                     
0001d00e  unlink                                     
0001d03e  DMA_startTransfer                          
0001d06c  __mspabi_negd                              
0001d09a  exit                                       
0001d0f6  DMA_getInterruptStatus                     
0001d122  __mspabi_divi                              
0001d122  __mspabi_remi                              
0001d14e  WaitForDRDY                                
0001d176  __mspabi_fixdi                             
0001d19e  UCS_clearFaultFlag                         
0001d1c4  __TI_zero_init                             
0001d1e8  usbReceiveDataPacketOnEP0                  
0001d20c  CdcIsReceiveInProgress                     
0001d22e  USB_disable                                
0001d250  USCI_B_SPI_transmitData                    
0001d272  __mspabi_mpyl_f5hw                         
0001d2d4  usbSetAddress                              
0001d314  DMA_setTransferSize                        
0001d332  memccpy                                    
0001d350  strcat                                     
0001d36e  usbGetInterface                            
0001d38c  usbGetInterfaceStatus                      
0001d3aa  IEP0InterruptHandler                       
0001d3c6  USCI_B_SPI_isBusy                          
0001d3e2  strchr                                     
0001d3fe  strcmp                                     
0001d41a  USB_connect                                
0001d434  USCI_B_SPI_receiveData                     
0001d44e  _abort_msg                                 
0001d468  USBCDC_handleSetLineCoding                 
0001d480  USB_resume                                 
0001d498  USCI_B_SPI_enable                          
0001d4b0  usbClearDeviceFeature                      
0001d4c8  usbSetDeviceFeature                        
0001d4e0  ADS126xSendADC2StartCommand                
0001d4f6  ADS126xSendADC2StopCommand                 
0001d50c  memchr                                     
0001d522  memset                                     
0001d538  printCommandPrompt                         
0001d54e  printError                                 
0001d564  __mspabi_divu                              
0001d564  __mspabi_remu                              
0001d57a  __mspabi_mpyi_f5hw                         
0001d590  usbGetConfigurationDescriptor              
0001d5a6  usbGetDeviceDescriptor                     
0001d5bc  USB_handleVbusOnEvent                      
0001d5e4  memcpy                                     
0001d5f8  usbGetConfiguration                        
0001d60c  usbSetControlLineState                     
0001d620  __TI_decompress_none                       
0001d632  strcpy                                     
0001d644  tolower                                    
0001d656  toupper                                    
0001d668  usbSetInterface                            
0001d67a  USBCDC_handleDataReceived                  
0001d68a  USBCDC_handleSetControlLineState           
0001d69a  USB_setEnabledEvents                       
0001d6aa  __mspabi_sral                              
0001d6ba  __mspabi_slll                              
0001d6ca  __mspabi_srll                              
0001d6da  SFR_clearInterrupt                         
0001d6e8  strlen                                     
0001d6f6  usbInvalidRequest                          
0001d704  usbRestoreInEndpointInterrupt              
0001d712  usbRestoreOutEndpointInterrupt             
0001d720  usbSendZeroLengthPacketOnIEP0              
0001d72e  USBCDC_handleReceiveCompleted              
0001d73a  USBCDC_handleSendCompleted                 
0001d746  __mspabi_fltid                             
0001d752  usbSetLineCoding                           
0001d75e  abs                                        
0001d768  __mspabi_slli                              
0001d772  __mspabi_srli                              
0001d77c  usbStallEndpoint0                          
0001d786  UCS_XT2Off                                 
0001d78e  USB_handleVbusOffEvent                     
0001d796  DMA_disableTransferDuringReadModifyWrite   
0001d79c  DMA_enableTransferDuringReadModifyWrite    
0001d7a2  USB_getVersion                             
0001d7a8  __mspabi_fltud                             
0001d7ae  __TI_decompress_rle24                      
0001d7b4  usbClearOEP0ByteCount                      
0001d7ba  usbStallOEP0                               
0001d7c0  USB_handleClockEvent                       
0001d7c4  USB_handleEnumCompleteEvent                
0001d7c8  USB_handleResetEvent                       
0001d7cc  USB_handleResumeEvent                      
0001d7d0  USB_handleSuspendEvent                     
0001d7d4  _system_pre_init                           
0001d7d8  C$$EXIT                                    
0001d7d8  abort                                      
0001d7dc  _nop                                       
ffffffff  __binit__                                  
ffffffff  __c_args__                                 
ffffffff  binit                                      
UNDEFED   __TI_INITARRAY_Base                        
UNDEFED   __TI_INITARRAY_Limit                       

[1194 symbols]
